:10000000A80B0020E1000000C1000000C1000000BA
:1000100000000000000000000000000000000000E0
:10002000000000000000000000000000C10000000F
:100030000000000000000000C1000000C10000003E
:10004000F5390000B90600004D3C0000E92600002B
:100050006126000099260000692A00003D2B00005F
:10006000C1000000F1010000110200003102000097
:10007000310800001D5A0000C1000000C10000004E
:10008000C1000000C1000000C1000000C10000006C
:10009000C1000000C1000000C1000000C10000005C
:1000A000C1000000C1000000C1000000C10000004C
:1000B000693B000025830000C1000000C100000072
:1000C000A023802170B50120592616258824DB0540
:1000D00049005E505D505C509A6802439A60F8E7B0
:1000E0001249134B10B599420BD2CA43D2180023C0
:1000F000920801320F489200C458CC500433934206
:10010000FAD10D480D4B98420BD2C1430024C918B7
:100110000023890801318900C218043314608B421E
:10012000FAD106F033F800F0E5FE10BD0000002023
:10013000000100203C92000000010020A8070020E0
:10014000002300B583B00193032802D9124803B0FD
:1001500000BD124B02301B6880000722C3401340D1
:100160006A46033213701378002B07D01378022BE2
:100170000DD01378072B06D00948E8E703F004FDFB
:1001800001900198E3E7074B01930198DFE703F043
:1001900035FD01900198DAE70197FFFF1402005046
:1001A0000297FFFF00805101F8B580234F46464675
:1001B0005B00C0B480460E000D0001240B4F994631
:1001C00003E00134AD194C450DD02900404608F03C
:1001D000F9F8831EBB42F4D8013C240620430CBC32
:1001E00090469946F8BD01204042F8E7FDFFFF0028
:1001F000012310B5044A91680B439360034B1869BF
:10020000DB68984710BDC046200001400001002077
:10021000012310B5044A91680B439360034B586A5D
:100220001B6A984710BDC046000011400001002025
:10023000012310B50C4A0D4C91680B439360A36ADF
:100240000133A362E36A002B07D0236B002B04D099
:10025000A36B013BA363002B00D010BDE36B206CAC
:100260009847636BA363F8E720001140000100206A
:100270000122034B5A649A64DA641A657047C046D7
:1002800000010020F8B546464F460400C0B40D00FA
:100290001600012800D170E0002852D0022827D093
:1002A000032849D14E490B6D012B00D096E04D4AF1
:1002B0009146D268002A00D090E048464A4FC36079
:1002C000BC46BF68B8462027404607436046876063
:1002D000464F3A60B8680343BB604B460A6303204D
:1002E0008A621D61FFF72CFF012860D8404824E096
:1002F0003B4B9C46DB6C012B00D06FE0394A116808
:1003000000296BD1384813608146806880461020F0
:10031000474638434F46B860364F3960B8680343A4
:10032000BB6063460220596151609560FFF708FF8A
:1003300001283CD82E4800E02F480CBC9046994636
:10034000F8BD274B5A6C012A48D1596D002945D177
:1003500025485A65876804313943284F81603C60DD
:10036000B96800200A43BA609C65DC661D67FFF728
:10037000E7FE01281BD81E48DFE7194B9A6C012ABB
:100380002CD15A6F002A29D108215867164887684E
:1003900039431B4F81603A60B96801202143B9603D
:1003A0001A609A67DD67FFF7CBFE01289ED9002D02
:1003B0009CD02900FFF7F8FE431C97D003021B0ACC
:1003C0007B60000EF306184338600020022EB4D183
:1003D0000F34E0B202F034FA0748AEE70948ACE760
:1003E0000001002080010020000200502000114088
:1003F0000297FFFF000011400197FFFF000001403E
:10040000200001400397FFFF70B582B0012800D1A2
:10041000C7E0002800D185E0022840D003287ED123
:100420007F48C66A002E00D0F7E001257D4CE562CA
:10043000C56A0135C56201960198002806DD6EE0A7
:100440000198013001900198002868DC019885002E
:10045000281880002018006B0028F1D10198850031
:1004600028180125800020180563019885002818A8
:10047000800020184163019885002818800020180A
:10048000816301998800411889006118CA63019A43
:10049000019891008A189200A418236440E06048F3
:1004A000856A002D00D0B8E00124C461846A01345B
:1004B000846201950198002831DC0198594C06E0CE
:1004C0000198013001900198002828DC01988500EE
:1004D00028188000201840690028F1D10198850073
:1004E00028180125800020184561019885002818EA
:1004F000800020188161019885002818800020184C
:10050000C161019988004118890061180A62019A45
:10051000019891008A189200A418636200E00020FC
:1005200002B070BD3E48056A002D76D101244461B9
:10053000046A01340462019501980028EFDC0198F7
:10054000384C06E001980130019001980028E6DC63
:1005500001988500281880002018806D0028F1D1AE
:1005600001988500281801258000201885650198CC
:100570008500281880002018C1650198850028187A
:1005800080002018016601998800411889006118CF
:100590004A66019A019891008A189200A418A366ED
:1005A000BEE71F4C656A002D37D1A061606A01303B
:1005B0006062019501980028B1DC0198194C06E0B1
:1005C00001980130019001980028A8DC019885006D
:1005D0002818800020580028F2D10198850028189A
:1005E00001258000255001988500281880002018DA
:1005F00041600198850028188000201881600199C9
:100600008800411889006118CA60019A0198910018
:100610008A189200A418236182E7034880E7C04645
:1006200080010020000100200497FFFF30B503285F
:1006300020D8114B8200D358104A8021944663443D
:100640001A6889050A431A600323FF220830C0B2E2
:10065000C2250340DB009A400949AD004C59944340
:1006600080229A40130023434B51012383400020F2
:100670000B6030BD0348FCE7D88600000000014055
:1006800000E100E00197FFFF03280CD8074A802112
:100690009446074B8000C358002063441A68C9057C
:1006A0000A431A6070470348FCE7C0460000014057
:1006B000D88600000197FFFF00B5094A83B0136890
:1006C0009B06DB0F0193082311680B431360054B56
:1006D0001B6B002B01D00198984703B000BDC046AA
:1006E00000400040800100208023A02210B55B0064
:1006F000D205D258FF3B134213D00B4A91680B43EB
:1007000080219360094A13688B43136007231468A0
:1007100018400302200006490840184310600020DA
:1007200010BD0448FCE7C0460002005000400040F5
:10073000FFF8FFFF0697FFFF4023034A11680B43B2
:100740001360024B18637047004000408001002096
:1007500010B509285ED8304B80001B589F460221F7
:1007600000202E4A13688B43136010BD07232B48CB
:10077000194004680B022100294A11401943016005
:100780000020F2E78023254A002011680B43136004
:10079000EBE78021214A002013688B431360E4E7D4
:1007A00040231E4A11680B43C02113601D4A890073
:1007B00050581D4B03408020000203435350022336
:1007C00000201360D1E74021144A002013688B43B6
:1007D00013608023134A3E39D150C6E710230F4AD5
:1007E000002011680B431360BFE710210B4A002063
:1007F00013688B431360B8E70123084A002011688F
:100800000B431360B1E70223044A002011680B4335
:100810001360AAE70548A8E7B08600000040004042
:10082000FFF8FFFF00E100E0FF00FFFF0597FFFF7B
:10083000044B10B51868044B1B68002B00D0984778
:1008400010BDC0461C000540B4010020F0B547466D
:10085000894B80B40D00184203D0884804BC9046F0
:10086000F0BD8A79072A00D9B5E0AB23D340DB0776
:1008700000D4B0E00B79032B00D9F7E04B79012BC2
:1008800000D9EAE0CB79062B00D9F1E0A023DB0503
:10089000DA688021002800D19FE089020A43DA60EB
:1008A000DC68774A2240DA60764A0426936801279A
:1008B0000B4393600222744BC4180F20A368334388
:1008C000A360A3681343A360EB79A1681840F023E9
:1008D000000199430143A160A879D03B3040411EFB
:1008E0008841E168400199430143E160AB791021FF
:1008F0001A40531E9A41E36812018B431343E3608D
:1009000008230322A879E16838409943C0000143D5
:10091000E160E1682B79914313401943E160FF21C5
:100920006A79E3683A409200B3431343E360236A71
:100930002A7A8B4313432362524B1A68D20752D54B
:100940005969524A0A405A614E4A966953693605B6
:100950009B01360F9B0F69D053699B019B0F012BA5
:100960007DD0711C4A4807F02DFD06002D6830002F
:10097000290007F027FD0F2307000340012B3ED974
:1009800080228021636A920513436362636A49058A
:100990000B436362BB1E98463E4B984511DD08250C
:1009A000636A1A436262626A3B4B134063626E1C65
:1009B0003100380007F08CFD02293ED9351E102D7C
:1009C000F5D14246636A1704380C1F0C3F040743F5
:1009D0006762002042E7314840E749020A43DA6093
:1009E000DC682F4A5EE71A6AD20317D51A685207E5
:1009F00040D5C0215A6989040A435A61A4E76D01B0
:100A0000B542BDD2626A274B070913406362626A2E
:100A1000214B13406362BB1E9846D2E759691B4ABB
:100A20000A40802149040A435A618DE703F0ACF87B
:100A3000711C07F0C7FC060098E70F23616A1A4A89
:100A40001D4011402B060D001D436562310038002A
:100A500007F0B8FC831E9846B3E71448FEE603F09F
:100A600097F8711C07F0AEFC06007FE71048F5E62A
:100A70001048F3E61048F1E6FFFFEFFF0298FFFF92
:100A8000FFFFFDFF0002005000000540FFFFFFFCDC
:100A900000805101FFFF0000FFFFFFEF0398FFFF01
:100AA000FFFFFEFFFFFFFFDFFFFFFFF00598FFFFE7
:100AB0000498FFFF0698FFFF0898FFFFF0B5012498
:100AC0004746260080B40227304B0E40C3185D68AD
:100AD0009046A54335435D605D684E08264076002C
:100AE000BD4335435D605D688E0826400237B60021
:100AF000BD4335435D605D68CE0826400437F6008F
:100B0000BD4335435D605E680D09B4466246204EC4
:100B10002540EF0216403E4310275E605E682D01BF
:100B2000BE4335434E098909214026408C014021AE
:100B30005D605D6810377601BD4335435D605D687B
:100B40008D4329002143596000280FD0C321114A49
:100B500089005058104B034080200002034353503B
:100B600080239B01136004BC9046F0BD4246C32025
:100B7000FF210A4B80001A60064B1A588A437F39BE
:100B80000A431A50802252011A60ECE70000054027
:100B9000FFF7FFFF00E100E0FF00FFFFB4010020CE
:100BA000224BF0B59C4603236044026B012513439E
:100BB00003634A78C46A531E9A411D4BD2032340F3
:100BC0001343C362C46A8B781A4E1A0623021B0AA7
:100BD0001343C3620A78C36A174C2A4012022340A7
:100BE0001343C3620A78C36A52082A405202334050
:100BF0001343C3620A78C76A9208104B2A409202D4
:100C00003B401343C362076ACA780D4B12023B4054
:100C1000134303620B7982681D402D0214402C435C
:100C2000846003691E400661F0BDC04600000540B7
:100C3000FF7FFFFFFFFDFFFFFFFEFFFFFFFBFFFF4B
:100C4000FF00FFFF30B50F241025114BDA68A243D7
:100C50000E3C2243DA60DA68AA43DA602022DD68BB
:100C60002A43DA60586099601A6914431C61BFF323
:100C70006F8F1A690649D207FBD40B6800205B0608
:100C800000D430BD40230A68024813430B60F8E7E4
:100C900000C000508188FFFF10B50F24124BDA68A6
:100CA000A243DA60DA680134A243DA60DA68103409
:100CB000A243DA60002258609A6018690132024348
:100CC0001A61BFF36F8F1A690748D207FBD4036814
:100CD0005B0603D4836800200B6010BD40230268CC
:100CE000134303600148F8E700C000508188FFFF0C
:100CF0000F21124BDA688A430D390A43DA60DA6849
:100D00000E318A43DA602022D9680A43DA60012270
:100D1000586019690A431A61BFF36F8F1A6907494E
:100D2000D207FBD40B6800205B0600D47047402339
:100D30000A68034813430B60F8E7C04600C0005040
:100D40008188FFFF0423054A51680B435360012348
:100D5000034A11680B4313607047C04600020050FD
:100D600000C000500121024A13688B431360704792
:100D700000C00050A022802330B5882059251624B9
:100D8000D2055B00D550D450D050D1580029F9D0AD
:100D900030BDC046F0B5474680B40C0082B0FF2895
:100DA00008D00130C5B2FF20152D22D902B004BCF5
:100DB0009046F0BD0223494A59259168E9380B4312
:100DC0009360A02280238821D2055B00A024D55007
:100DD000D050D150D658E405002EF7D0FFF7B2FF1F
:100DE000F8204002FFF784FF0123A2681343A360A9
:100DF000FEE7012D0CD109296DD90B1C182900D94A
:100E00001823DCB2364B1B190A3B1B78354A13609A
:100E1000354F785DC0B28442C8D08821A02280239B
:100E2000592616208846D2055B004146D650D05040
:100E3000D150D1580029F8D0802180232B4A890134
:100E4000D150FFF77FFFF823DB01EE18B60001A9B0
:100E50003000FFF721FF1022019B904623409C4267
:100E600007D131E001235B429C46E0444346002B1E
:100E70001AD0F8204002FFF73BFFF82001A94002FA
:100E8000FFF70AFF019B0133ECD17C55F8250024C4
:100E90006D02174B395D9C46280061440134FFF711
:100EA000D1FE0435152CF4D101A93000FFF7F4FE72
:100EB000019BDCB2FFF756FF80220C4B92011A60B7
:100EC00002F080FD200071E7094B3000E11801912C
:100ED000FFF7B8FEE8E730230A2497E70041005007
:100EE000C88A000010000440F002002000E100E089
:100EF0000000FFFFF0B54D4644465F465646234B83
:100F0000F0B4234C23492360234B24480B60244B2B
:100F1000244A0360244B254D1360254BF1B01D601E
:100F2000802585600020A06088600A2191603822B9
:100F30009A60A02280235924D2055B0016307E31AE
:100F4000D450D050D150D558002DF9D00122194B92
:100F500019680A431A60D968164AC907FBD5116A8D
:100F6000154B164C0B4013620C2323602368DB07E0
:100F700026D4C823012122685B0852082260226817
:100F80001A431142F7D0023B1BE0C046FFCF0000DE
:100F90000040005040400050F0FF000080400050F2
:100FA000FFF70000C0400050CF5D0000D50F0000EB
:100FB0000041005000020050FFFFF7FFD002002068
:100FC000C623C0252268F449023A2D0252022A4360
:100FD0000E6A1343DA05D00D720A520202439B04D3
:100FE0000A62DB0E086A5A02EC4B034013430B62A1
:100FF0000B6A1D430D620A6AE94B13400B620A6AD1
:10100000E84B13400B620B00D968E34A4907FBD554
:10101000072113698B43190002230B431361D36823
:101020001B0603D58023D1680B43D36005F068F815
:1010300002F0AEFD2060FFF785FEF8200AAD290022
:101040004002FFF729FED84B0A9A9A4201D000F0DD
:10105000F8FCF82600242900D44B760203933000D4
:10106000FFF71AFE0A9B039ADBB2135501340AA953
:101070000436152CF3D10D00CD4B0493CD4ECE4B41
:10108000F9273400984629007F023800FFF704FE54
:101090000A9B04371A0E22701A0C62701A0AA27088
:1010A000E3700AA904344745EFD133780D00FF2BD4
:1010B00003D1DF3B3370002373702900BF48FFF773
:1010C000EBFDFFF74FFE0023BD4A0124137092226F
:1010D000120694460A9BBB4D1B021B0A2B602B6811
:1010E000832263442B60B84B02211C709B46032370
:1010F00000200093002307F0A7F8B44AB44B516ACC
:101100000B40802189000B435362B24B1C6007F0F7
:1011100047F9B14B1B699B0702D40423039A13714F
:10112000AE4B1B691B0704D4042203994B799343EC
:101130004B71AA4B1B69DB0608D4082303994A7933
:10114000134304224B714B7993434B71A34B1B699F
:101150009B0608D4082203994B7993434B710423CF
:101160004A7913434B71039B5B791B0704D54023DA
:101170009B4A91680B4393609023994AA0249168FD
:1011800004200B4393600023984642461F21954B51
:10119000E4051A70944B81461A702B68934ADBB2AF
:1011A0001370934A934E137013780B401370924A46
:1011B000924B11680B4003210B431360904A8A46FF
:1011C000904B11680B40C02109010B438021136033
:1011D000E36849020B43E360E368724A1A40E26045
:1011E0006D4A93680B439360874B996801439960FC
:1011F000022198680143F0209960996881439960C1
:10120000D968D03881435046D960D96801434846EF
:10121000D960D9688143D960D9688143D960196A96
:10122000FB30814319625169784B0B4053619769D8
:1012300002F0AAFC802233689205134380223360B7
:10124000336852053F0513433F0F3360791C07F0A5
:10125000B9F86F4907F0B6F83168831E1B041A0C01
:101260000B0C1B0413433360226B6A4BC3271340E0
:1012700008222363236B012193432363226B664B74
:1012800000201A402263226BBF0013402363634A8D
:10129000FFF714FCFF22624C1420E359012693430C
:1012A0001A0080231343E35101F0CAFA5D495E4BF3
:1012B00080200B6053460B7143464B718E71CB718E
:1012C0000A232A6840031343DBB20B72FFF7BEFA0E
:1012D000434608A98B70052380200B7043464003CA
:1012E000CB700B714E70FFF75BFC80200022012158
:1012F0004003FFF7E3FBE2594C4B002113408022EF
:10130000D2011343E351062001F016FA0221032013
:1013100001F0F8F90321032001F0F4F94246444BAF
:101320000D201A7001F08CFA0E2001F089FA2A4B78
:10133000404AC025DA61052252429A614B46AD000F
:10134000236062593C4B01211340635100223B4B07
:10135000032001F00BFAC022635912061B021B0A7C
:101360001343635101F072FF152001F069FA344B09
:101370000CAC0D9343466370434600210F9300204D
:1013800032330E93267002F0E9FA2100002002F0B9
:1013900017F80121002055E000020050FFC1FFFFB7
:1013A000FFFFFBFFFFFFFEFFA500FFFFF002002095
:1013B000C88A00005C05002018F20100FC0F100034
:1013C000AE020020B40200201D03002000000E40E9
:1013D000FFFCFFFF1C000050C040005000410050C7
:1013E00080400050A4070020B202002050050020D9
:1013F00049040020240005403C000050FCFCFFFF95
:1014000030000050F3F3FFFF00000540FFFFFFFC3A
:1014100090D00300FFF7FFFFFFFBFFFF6D590000B7
:1014200000E100E0D402002020A10700FF00FFFF40
:101430008205002004000400FFFF00FF05410000BA
:101440003075000002F034FA0121002001F058FF4D
:10145000039930234A78092A08D94A787523182A2B
:1014600004D84B78049A0A3BDBB2D35C0025CE4A01
:10147000CE4C1360CE4B1D70FEF7FAFE20230121E7
:10148000A26888461343A360CA4B47461D609A680A
:101490000A43C0219A60C84A49055A60186808433F
:1014A000186080201E68C00506431E600423A668DD
:1014B0003343A360C14B1D609E683E439E605A60EB
:1014C0001A68C22611431960FA211A68890002437A
:1014D0001A6001200122FEF7D5FE0120FFF7D4F8A3
:1014E000B74F0120FFF7A2F8B6000023B54A01214B
:1014F0000120FEF789FFBA59B34BB4491340C0220B
:1015000012021343BB5100220220FEF7BBFE022051
:10151000FFF78CF80023AE4A01210220FEF774FF8A
:10152000BA59AC4B01211340C02212041343BB51E2
:10153000002002F06FFA03236269062013436361FF
:10154000FFF7D2F8A448FFF7F7F800210220FFF7D1
:10155000FFF800210020FFF7FBF802F033FA9F4B61
:101560001D709F4B1D805B461B78002B05D0802390
:101570008F4A137042469B4B1A70002307930693C1
:10158000059380330493984B59269A46974B50AC59
:101590009B4630AB9946964B9846A0228023162551
:1015A0008820D2055B00D650D550D050D1580029A4
:1015B000F9D001238F4A11680B43136002F002FA3D
:1015C0007B4B1B785BB2002B03DBFA238A4A5B0060
:1015D000136053461B685B0730D5A0228023162575
:1015E0008820D2055B00D650D550D050D158002964
:1015F000F9D0FFF7A7FBF920F9274002FFF778FBA6
:101600007E4D7F0229786B7809061B04C918AB78D8
:1016100038001B02C918EB780437C918FFF712FB12
:10162000774B04359F42EDD1FFF79CFB02F0CAF9DE
:10163000534604221B689343524613605B461B6863
:101640009B0536D55B461A686E4B13405A461360AD
:10165000574B1B785BB2002B01DA00F086FD0023AC
:10166000694A13700023694A13805B461B689B021A
:1016700001D500F0FDFB0825654B0A201978C9B299
:10168000FFF788FB624B039F1B780B20DBB2FB72DA
:10169000604B19782943C9B2FFF77CFB5D4B1B787F
:1016A0002B43DBB23B735B461A685B4B13405A46D5
:1016B00013605A4B1B78032B00D129E23C4B049A50
:1016C0001B789A420AD03A4B1B785BB2002B01DAA6
:1016D00000F016FD364B1B78DBB2049343461B88A3
:1016E000002B00D193E10023424613804C4B1A6B30
:1016F000D20700D48BE10122196B0A431A635246C8
:101700001268D20301D500F046FD1A68920307D58E
:101710002820324A12781968530006AA1218D152AA
:101720003F4B5A68920304D52C4A127859685300EB
:10173000E1523B4AD3699B030AD5284B27481B78C3
:10174000DBB2591CC9B201704946D2695B00CA526A
:101750003F22224B1B781340204A1370FA22304B51
:1017600012011B689BB2934206D9114B1B785BB2E6
:10177000002B01DA00F09EFD534620221B68294908
:1017800093435246136007220B6800209343063AA6
:1017900013430B608021224A0901136A0B43136231
:1017A000002110AA44E0C04610000440000200508E
:1017B0008605002020001140FFFF000000000140CE
:1017C00000E100E0F1410000FF00FFFFF82A000007
:1017D00099480000FFFF00FFF56000002E03002085
:1017E0008405002074050020900700207C0500205F
:1017F0004E05002000400040E00200205C05002073
:1018000018F20100FFFDFFFFAE020020B002002031
:101810002F0300208C070020FFFFCFAFA40700207C
:1018200000000E4030000E400232401891450CD0AE
:1018300013881D1C8B4200D20D1CA9B28D08AB422F
:10184000F2D30232C0189145F2D13E2106F0BAFD22
:10185000039AC3B20793137D984201D2107DC0B2A0
:10186000039D64212B7DC01AAF235B00584306F013
:10187000A9FD8D4B1B689C46059360448A4B40082C
:101880001860FA232A799B005343984202D200231E
:10189000864A137053461B685B0602D50023834AB1
:1018A00013708022824B1B69134001D17F4A137051
:1018B000039D7E4BAA781B789A424FD2002280204B
:1018C0007A4B7B491A708B6883438B60402379493C
:1018D000886803438B60032377490B707749023B89
:1018E0000B705B4680211B68C9030B4359460B6094
:1018F000734B73491B780133DBB20B70714B724928
:101900000B806F4B1B78052B01D800F04CFCAB7A99
:101910006E49DBB20B706A4B1A7000236C4A13805D
:101920005B461A686B4B13405A4613606A4B1B8820
:10193000002B11D1694B684A13802023684A9168B3
:101940000B43936053461B685B0305D50122654B2F
:101950001A601423644A1360534B18680F2801D986
:1019600000F010FC614BC0B218704B460022198881
:10197000023352189C42FAD1524B92095A435C4BA3
:10198000120B9A4201D900F0F5FB64204042424319
:10199000584BAF21D01806F015FDC3B20593502B5C
:1019A00001D800F018FE8021414A434893688B43D8
:1019B000936040233F498A681A438A60022202707A
:1019C000886803438B605B4680211B68C9000B431A
:1019D00059460B60394B1A70374B1A7000233C4A3A
:1019E00013800A683B4B13400B6006AAD32394462E
:1019F00000225B0063441988023B52189C42FAD1D2
:101A0000FA2392095B005A43120BD3B206935B464A
:101A10001B68DB0700D4C0E50F22374B1B789343CC
:101A2000C02B00D15AE30F22334B5B789343E02B5A
:101A300000D155E25B4601221B6893435A4613606E
:101A4000ABE529002D48FFF727F9F8200A9B2C4A1F
:101A5000DBB24002F826137503920024FFF748F921
:101A6000A522284B76020493039B30001A55195D7A
:101A7000254B04369C4661442960FFF7E3F8631C5C
:101A8000142B04D0049A1C0010329A5CECE7039BE0
:101A9000197D1D4B9C461D4B6144E0188000296058
:101AA000FFF7D0F8FFF7EAFAB80100205905002047
:101AB00000400050C0400050AE02002086050020CB
:101AC00058050020881300002C0300207805002012
:101AD000B0020020FFFFFFBFBA020020DC050000BB
:101AE0008040005070420050540500201C0300202C
:101AF000DE020000B81E01000803002050F00100C3
:101B0000F0020020C88A00000000FFFF017C0000F6
:101B1000E84B1A78E84B1B789A4200D0C7E15B4645
:101B20001A6880239B04134069D1524612685203FD
:101B300065D5524601211268114260D052461268A2
:101B40008A4351460A60DD4A1278002A57D05A4625
:101B500080211268C9040A4359460A60D84AD84805
:101B60001278D2B2511CC9B201700621D5488154F5
:101B7000D34AD3481278D2B2511CC9B201700521A0
:101B8000D0488154CE4ACE481278D2B2511CC9B244
:101B90000170CC498B540378DBB25A1CD2B202706C
:101BA000C94AC9481278D2B2511CC9B20170C5499C
:101BB000CA54C34BC2491B78DBB25A1CD2B20A705A
:101BC0008622C049CA54BE4BBD491B78DBB25A1CA1
:101BD000D2B20A700422BB49CA54B94BB8491B7827
:101BE000DBB25A1CD2B20A70B44AB6491278D2B2E9
:101BF000CA545B461A68B54B13405A4613605346A5
:101C00001B685B0300D4CCE05B461A688023DB04CE
:101C1000134000D0C5E05A461268120273D55A46E6
:101C20001168AB4A0A4059460A60AA4A127852B271
:101C3000002A01DA00F05FFCA14AA1481278A24D07
:101C4000D2B2511CC9B201700A219E4881549C4AEB
:101C50009B481278D2B2511CC9B20170092199482F
:101C60008154974A96481278D2B2511CC9B2017079
:101C700094498B540278D2B2511CC9B20170924976
:101C80000978C9B2481CC0B228708E4881548C4A69
:101C90008B481278D2B2511CC9B20170B221894866
:101CA0008154874A86481278D2B2511CC9B2017059
:101CB000012184488154824A81481278D2B2511C51
:101CC000C9B201707F498B540278D2B2511CC9B29B
:101CD00001707C498B540278D2B2511CC9B2017098
:101CE00078498B5403787749DBB25A1CD2B2027020
:101CF0000222CA5469460378097DDBB25A1CD2B26B
:101D00000270704AD15453461B685B0149D5534653
:101D10001A686E4B6A49134052461360684B6A4812
:101D20001B78DBB25A1CD2B20A7005226549CA542C
:101D3000634B63491B78DBB25A1CD2B20A7004228F
:101D40006049CA545E4B5E491B78DBB25A1CD2B262
:101D50000A7000225B49CA54594B59491B78DBB2BF
:101D60005A1CD2B20A70584A1278D2B2511CC9B267
:101D700001705449CA54524B1B785149DBB25A1C6A
:101D8000D2B20A70B0224F49CA544D4B4C491B780D
:101D9000DBB25A1CD2B20A704E4A4A491278D2B209
:101DA000CA544C4B049A1B789A4200D196E4494B92
:101DB0001B785BB2002B00DA07E2464B1B78DBB2E4
:101DC000049353461B685B0300D487E45B46802280
:101DD0001B68D20413435A461360394B38491B78A9
:101DE0003948DBB25A1CD2B20A7005223549CA54AE
:101DF000334B33491B78DBB25A1CD2B20A7004222F
:101E00003049CA542E4B2E491B78DBB25A1CD2B231
:101E10000A7000222B49CA54294B29491B78DBB28E
:101E20005A1CD2B20A70284A1278D2B2511CC9B2D6
:101E300001702449CA54224B1B782149DBB25A1C39
:101E4000D2B20A70B0221F49CA541D4B1C491B78DC
:101E5000DBB25A1CD2B20A701E4A1A491278D2B2A8
:101E6000CA545B461A68194B13405A46136035E44E
:101E7000194B0C2019780825C9B2FEF78BFF0122F7
:101E8000154B039F1B780D20DBB27B73134B1B7824
:101E90009343124A137011782943C9B2FEF77AFFAF
:101EA0000E4B1B782B43DBB2BB73FFF7FCFB04F03C
:101EB000B5F9A4E6A50700209807002094070020A4
:101EC000EC0200204C0400204D050020FFFFFFFB2A
:101ED000FFFF7FFF860500202F0300208C070020D6
:101EE000DF4B033A5B7813400C2B00D0A2E5DC4BB0
:101EF000DB4A5B7892788021D0B25A461268C905D5
:101F0000DBB20A4200D18FE1D54BDB783E2B0BD000
:101F10000523D44A13700023D34A13805B461A6802
:101F2000D24B13405A461360CD4BDB78083BDBB2F3
:101F3000F72B00D97EE5CE4A9B00D3589F46079DDC
:101F400013202900FEF726FF039B1D7572E5C44B85
:101F50000320D9780B002821773B5943C9B2FEF7FB
:101F600019FF67E5BE4B0220D9780B0014216D3BA9
:101F70005943C9B2FEF70EFF5CE5B94B0920D97889
:101F800064398B00C9184900C9B2FEF703FF51E557
:101F90005B4680221B68520513435A46136009238F
:101FA000B04A1370B34BB04A138043E55B461A68DE
:101FB000B14B102513405A46039F13607979A9430A
:101FC0000420FEF7E7FE7B79AB437B7132E55B468D
:101FD00080221B68520413435A461025039F136046
:101FE00079792943C9B20420FEF7D4FE7B792B43CB
:101FF000DBB27B711EE55B4681221B68CBE75B464B
:102000001A689E4B039F13405A4613607979202526
:10201000D5E75B4680221B68520313435A46039F51
:10202000136079792025DCE7039F08257979C6E7D5
:102030000823039D042069791943FEF7ABFE0423AE
:10204000697904209943FEF7A5FE04236A791343B6
:1020500008226B716B7993436B71EBE4039F04254A
:102060007979ACE70425039F042079792943C9B223
:10207000FEF790FE0397797908270420B943FEF70D
:1020800089FE039A53791D43EDB255715379BB43D1
:102090005371CFE4039F0125797990E7039F0125D0
:1020A00079799EE76E4B0320D9782839C9B2FEF7BB
:1020B00071FEBFE46A4B0820D9781E39C9B2FEF719
:1020C00069FEB7E4664B0020D978C9B2FEF762FE1C
:1020D000B0E43E21FF20FEF75DFEABE4604B604ABA
:1020E0009B78DBB25370D378DBB293701379DBB299
:1020F000D3705379DBB213719379DBB2537192E4ED
:102100005F4B1B88002B01D0FFF7E8FA20215D4AC6
:102110005D4893688B4393601C3903695A4A19429E
:10212000FBD180235949886803438B6040230220F8
:1021300091689943916056498A6882438A60039AFC
:102140005449D27852000A805246126813435246CC
:1021500013600022504B1B78DBB2049310AB1A8043
:1021600002339945FBD1FFF7B9FA05233D4A1370B5
:10217000FFF778FA5B461B685B0500D592E1002308
:10218000059332E4CF2815D883080C33434ADBB2D9
:102190001370FFF7EAFB53461A68414B134052464F
:1021A0001360FFF7C6FA039B3E4A5B7ADBB21370FB
:1021B000FFF7B3FB3C4B984200D986E10309333368
:1021C000364ADBB21370FFF7D0FB20212D4A93680B
:1021D0008B4380219360354AC90413680B438021E7
:1021E00013601368C9050B4313608023274A916865
:1021F0000B439360402324498A689A438A60039A78
:102200002449D27852000A8052461268134352463B
:102210001360FA23264A5B001360002210AB1A8079
:1022200002339945FBD1C8E5032213401B021B185A
:10223000062B01D0FFF7FEFB094BDB783E2B01D0CC
:10224000FFF7F8FB0B4B084A13805B461B68054AF7
:1022500019435B46196008231370FFF7EBFBC04678
:1022600008030020AE020020B0020020FFFFFFBFE5
:10227000E886000030750000FFFFFFFEFFFFEFFF64
:10228000E402002080400050C04000500040005058
:1022900000410050A0020020860500201C03002001
:1022A000FFFFFEFF78050020FF0400002000114022
:1022B000E002002053461A68202313435246039934
:1022C00013608B78CA4A1380534640221B681A4217
:1022D0000FD053461B68934352461360C44ACB78D1
:1022E00012885B00D318C24A9BB213800023C14AF4
:1022F00013800420C04BC1499C46C14B62468025D7
:102300009268AA436546AA6040258A682A438A6083
:102310000A69BA4D1042FBD16246802792683A435F
:102320006746BA604027AA68BA43AA604246128844
:10233000002AFBD04246002507271580B14D2A68A8
:10234000BA43063F3A432A6080251A6A2D012A4380
:102350001A621D6BAA4AED07FBD50127156B3D4399
:1023600000271563A84D2F701568A84FADB2BD4268
:1023700035D80727A34D2D68BD43063F3D43A14FE8
:102380003D608027156A3F013D4315621D6B9C4AE5
:10239000ED07FBD50127156B3D43156315689B4F72
:1023A000ADB2BD421BD80727964D2D68BD43063FF1
:1023B0003D43944F3D608027156A3F013D431562C0
:1023C0001A6B8F4DD207FBD501272A6B3A432A633C
:1023D0002A688E4D92B2AA4201D8FFF7CDF9844AFD
:1023E0001288002A8AD1FA22854B12011B689BB2FF
:1023F000934201D8FFF7C0F980217F4A93688B434D
:10240000936040237D4A91680B4393600323804A85
:102410001370804A023B13705B4680221B68D20314
:1024200013435A4613607C4B7B4A1B780133DBB263
:1024300013707A4B7A4A1380774B1B78052B00D8A0
:10244000BDE0039A937A002B00D1BEE0937A754ADF
:10245000DBB213700023704A13700023724A13809A
:102460005B461A68714B13405A461360704B1B88C9
:10247000002B01D0FFF780F96E4B6D4A13802023AB
:102480006D4A91680B43936053461B685B0301D40C
:10249000FFF772F90122694B1A601423684A13602E
:1024A000FFF76AF9002305935B461A68654B1340F2
:1024B0005A4613600023574A1370634A1278032A5E
:1024C00014D0534A1370FFF790FA604B984206D825
:1024D00083096C335E4ADBB21370FFF746FA030AD6
:1024E000553B5B4ADBB21370FFF73FFA484A0633AD
:1024F0001370FFF77AFA20204F49564D8A688243BD
:102500008A60554A54481278D2B2511CC9B201703F
:102510000A2152488154504A4F481278D2B2511C75
:10252000C9B2017009214D4881544B4A4A4812787A
:10253000D2B2511CC9B2017048498B540278D2B250
:10254000511CC9B2017043490978C9B2481CC0B2D4
:10255000287042488154404A3F481278D2B2511CF8
:10256000C9B20170B2213D4881543B4A3A481278C1
:10257000D2B2511CC9B20170012138488154364A87
:1025800035481278D2B2511CC9B20170684633493D
:10259000007E8854304A30481278D2B2511CC9B2F9
:1025A00001702E498B5403782C49DBB25A1CD2B2ED
:1025B0000270274A1278D2B2CA54FFF793FB039BEA
:1025C000184A5B7ADBB2137047E7039B154A5B7AC4
:1025D000DBB213703EE75B461B685B0501D4FFF777
:1025E00004FA059B402B01D9FFF7FFF95CE7C046D1
:1025F000A2070020A002002000400050C040005070
:1026000000000E4030000E40590500209F0F0000D2
:10261000AE02002086050020580500208813000027
:102620002C03002078050020B0020020FFFFFFBF30
:10263000BA020020DC0500008040005070420050CB
:1026400054050020FFFBFFFFA4070020FF1400003B
:102650001C0300204D050020EC0200204C0400204B
:1026600000B50A4A83B0136A0093094B196A0191B5
:1026700000991162019A1A62064B1B68002B02D066
:1026800000980199984703B000BDC0460040005033
:1026900040400050DC01002010B50C240E4884B0EE
:1026A000036A0E4901930B6A0D4A0293136A03935E
:1026B000029BA3430293019B0362029B0B62039B59
:1026C0001362084B5B68002B03D001980299039AB0
:1026D000984704B010BDC04680400050C040005034
:1026E00000410050DC0100200822044B10B51A62A2
:1026F000034B9B68002B00D0984710BDC040005092
:10270000DC0100200A4B80019C4682B060440190AD
:102710000198019B1A6801238B4013430360202317
:102720000020044A11680B43136002B07047C04692
:10273000144000508041005010B50F2810D80F24CD
:10274000084B20401A68A2431043186001201A6801
:1027500001400F308243002009011143196010BD70
:102760000148FCE7804100500189FFFFF0B52F4C84
:1027700083B00194002926D1019D019906000C68BF
:1027800001210F001036B74081403C432C60284C9B
:102790000194019C002A21D1019A12688A43226087
:1027A000022821D0C0218020224A89009360224A39
:1027B000000653581B021B0A03435350082313609F
:1027C000002003B0F0BD01291BD0022920D0012137
:1027D000174C81400194019C002ADDD0019A1268B7
:1027E000114321600228DDD1C021134A89005058CD
:1027F000124B034080200004034353500423136012
:10280000DEE78140019D019C24680C432C60BEE7FB
:102810000124019E019907000D68210010378140B5
:10282000BC400C432C433460B1E7C046DC40005050
:10283000D8400050DC01002000E100E0FFFF00FF75
:1028400030B51D2800D9E7E0744A8300D3589F466D
:10285000FF2273490B681B0C1B0413430B60FF2200
:10286000704900200B681B0C1B0413436E4A0B605D
:1028700011686E4B0B40802109010B4313601168F6
:102880006B4B0B40C0210B436A4913600A686A4BCB
:102890001340302213430B6030BD6649644B0A6815
:1028A00000201340C02213430B60F5E700235D4A6C
:1028B00000201360614A1360594A13605A4A13603A
:1028C0005C4A1360E8E7584A5D4B116800200B40F2
:1028D0008021C9010B431360DEE7534A564B116850
:1028E00000200B40C02189010B431360D4E7534AF9
:1028F0001168544B00200B40F02109020B43136078
:10290000CAE7484AF4E701231D00C41CA540053866
:1029100083404A4900200A68AA4313430B60BBE77F
:102920004149494B0A6800201340042213430B60BD
:10293000B2E73D493D4B0A6800201340082213438B
:102940000B60A9E73849414B0A6800201340102268
:1029500013430B60A0E734493D4B0A680020134045
:10296000202213430B6097E7344A3A4B116800204A
:102970000B40802149000B4313608DE72F4A364BF3
:10298000116800200B40802189000B43136083E70E
:102990002549324B0A680020134003221343214A81
:1029A0000B6011682E4B0B40C02109010B431360D3
:1029B00072E7224A2A4B116800200B40C02109010E
:1029C0000B431360174A254B11680B40C021890047
:1029D0000B43136060E703231138400004001D001F
:1029E000083C8340A5400E4900200A681343AB43CE
:1029F0000B6051E70F490A68192806D0184B0020D0
:102A000013400C2213430B6046E7144B0020134085
:102A1000032213430B603FE712483DE7F08A0000B2
:102A200038000050300000503C000050F7F7FFFF26
:102A30003F3FFFFF40000050CFCFFFFF340000506A
:102A4000BFBFFFFF0F0FFFFFFBFBFFFFEFEFFFFF1E
:102A5000DFDFFFFFFEFEFFFFFDFDFFFFFCFCFFFFD2
:102A6000F3F3FFFF0189FFFF01222E4B70B51C68B5
:102A7000224205D01A602C4B1B68002B00D09847CF
:102A80000223234206D0274A1360274B9B68002B62
:102A900000D098470423234206D0224A1360224BD9
:102AA0001B69002B00D098470823234206D01D4AFB
:102AB00013601D4B9B69002B00D098471B4B1C4A91
:102AC0001D681468EA0608D519681A4A0A401A608F
:102AD000154B5B68002B00D09847EB0209D5134AD1
:102AE000154B11680B4013600F4BDB68002B00D0B7
:102AF0009847E30609D50E4A0E4B11680B40136048
:102B0000094B5B69002B00D09847E30209D5084ABE
:102B1000094B11680B401360034BDB69002B00D09D
:102B2000984770BD44000440E80100205000044074
:102B3000540004401F000F000F001F0001222E4B05
:102B400070B51C68224205D01A602C4B1B6A002B02
:102B500000D098470223234206D0274A1360274B10
:102B60009B6A002B00D098470423234206D0224AB8
:102B70001360224B1B6B002B00D098470823234285
:102B800006D01D4A13601D4B9B6B002B00D098474D
:102B90001B4B1C4A1D681468EA0608D519681A4AB6
:102BA0000A401A60154B5B6A002B00D09847EB0275
:102BB00009D5134A154B11680B4013600F4BDB6AA4
:102BC000002B00D09847E30609D50E4A0E4B11683A
:102BD0000B401360094B5B6B002B00D09847E3025E
:102BE00009D5084A094B11680B401360034BDB6B96
:102BF000002B00D0984770BD44001440E80100202D
:102C000050001440540014401F000F000F001F001C
:102C100001230B4030B51C0002231940172800D9AE
:102C20000BE1884D8300EB589F46002C07D0864867
:102C3000864B046823408024A402234303600029B8
:102C400007D08149824B086803408020C0020343BB
:102C50000B60804BDA631AE001237F49086C034361
:102C60000B647C4B1A60C1217C4A890050587C4B14
:102C7000034080200004034353504023136030BDC1
:102C800008237849086C03430B64724B9A63C12193
:102C90008020724A8900535800061B021B0A034316
:102CA000535080231360EAE7002C06D06E4C6F4B24
:102CB00020680340022003432360002906D06A48AD
:102CC0006B4B01680B4004210B430360614B5A605E
:102CD000C9E7002C07D064485C4B0468234080247B
:102CE000A40223430360002907D05F49584B0868BA
:102CF00003408020C00203430B60564BDA60B2E70A
:102D0000002C06D05B4C594B206803400220034343
:102D10002360002906D05748554B01680B40042119
:102D20000B4303604B4B5A619DE7002C07D0514881
:102D3000464B046823408024A402234303600029F7
:102D400007D04C49424B086803408020C00203432F
:102D50000B60404BDA6186E7002C07D046483B4BBE
:102D6000046823408024A40223430360002907D081
:102D70004149374B086803408020C00203430B6081
:102D8000344BDA6283E7002C06D03B4C374B20688B
:102D90000340022003432360002906D03648344B09
:102DA00001680B4004210B4303602A4B5A626EE713
:102DB000002C06D0244C2D4B2068034002200343F6
:102DC0002360002906D02048294B01680B400421CC
:102DD0000B4303601F4B5A6359E708231E49086CD5
:102DE00003430B641B4B9A613DE702231A49086CAD
:102DF00003430B64174B9A6035E704231649086CAC
:102E000003430B64134B1A612DE702231549086C29
:102E100003430B640F4B9A6239E704231149086C92
:102E200003430B640B4B1A6331E701230D49086C14
:102E300003430B64074B1A6229E7430700D412E7E8
:102E400025E7C046688B0000540014400F000D00B9
:102E50000F000B00E80100200000044000E100E04A
:102E6000FFFF00FF00001440500004400D000F0061
:102E70000B000F00540004405000144017280BD8DA
:102E8000514B80001B589F46504A514B11680B40D4
:102E9000136000224F4BDA63704701224E490B6CDE
:102EA00093430B644D4B1A6000224A4B1A60F3E7C0
:102EB000022249490B6C93430B64484B1A60002271
:102EC000444B9A60E8E7042243490B6C93430B643C
:102ED000424B1A6000223F4B1A61DDE708223E494F
:102EE0000B6C93430B643D4B1A600022394B9A6183
:102EF000D2E701223A490B6C93430B64394B1A60B9
:102F00000022344B1A62C7E7022235490B6C934307
:102F10000B64344B1A6000222E4B9A62BCE70422E9
:102F20002F490B6C93430B642E4B1A600022294BE4
:102F30001A63B1E708222A490B6C93430B64294BAF
:102F40001A600022234B9A63A6E7274A274B116891
:102F50000B40136000221F4B5A609DE7224A1C4B16
:102F600011680B40136000221A4BDA6094E7204A84
:102F70001E4B11680B4013600022164B5A618BE701
:102F80001B4A134B11680B4013600022114BDA618E
:102F900082E7184A154B11680B40136000220D4B55
:102FA0005A6279E7134A0A4B11680B4013600022FA
:102FB000084BDA6270E7054A0C4B11680B4013604E
:102FC0000022044B5A6367E7C88B0000540014408A
:102FD0000F000900E8010020000004404400044004
:102FE00000001440440014405000044009000F0049
:102FF0005400044050001440172808D81F4A83008A
:10300000D3589F461E4A1F4B11680B4013607047F0
:10301000012383401C4A1360F9E7012304388340ED
:103020001A4A1360F3E71A4A1A4B11680B401360EF
:10303000EDE7174A134B11680B401360E7E7164A98
:10304000144B11680B401360E1E7134A0D4B1168F4
:103050000B401360DBE7114A0E4B11680B40136005
:10306000D5E70E4A074B11680B401360CFE7044ABF
:10307000084B11680B401360C9E7C046288C00005C
:10308000540014400F001F0044000440440014404A
:10309000500004401F000F00540004405000144032
:1030A00017283DD81F4A8300D3589F461E4B586DA2
:1030B000C002C00F70471D4B1A68012383401800DF
:1030C0001040431E9841F5E7194B1A68031F012071
:1030D00098401040431E9841ECE7164B186DC0060F
:1030E000C00FE7E7134B186DC002C00FE2E7114BAA
:1030F000586DC006C00FDDE70E4B586DC002C00F03
:10310000D8E7094B186DC006C00FD3E7064B186D02
:10311000C002C00FCEE7044B586DC006C00FC9E710
:103120000020C7E7888C00000000144044000440E1
:1031300044001440000004401038C0B2072833D8BF
:103140001A4B80001B589F46194B586D06290DD00D
:103150000006C00F7047164B586D062912D00002AA
:10316000C00FF7E7134B586D0629F1D14006C00F89
:10317000F0E7104B186D0629EAD1F7E70D4B186DF3
:103180000629ECD14002C00FE4E7094B186D06296F
:10319000DED1EBE7064B186D0629E0D1F2E7054BCF
:1031A000586D0629DBD1EDE70020D3E7E88C00005D
:1031B00000001440000004401038C0B207280AD8AC
:1031C000194B80001B589F46184A062917D01168D2
:1031D000174B0B4013607047144A062907D011683B
:1031E000144B0B401360F6E7134A0629F7D1116818
:1031F000124B0B401360EEE70F4A0629E7D1116826
:103200000F4B0B401360E6E70E4A0629E7D1EEE7C5
:103210000C4A0629DBD1F2E70B4A0629DFD1E6E7A3
:10322000094A0629D3D1EAE7088D0000540014406A
:103230000F008F008F000F00500004404F000F0060
:103240000F004F005400044050001440F021084A81
:10325000090413680B43C0211360064B89031A68E5
:103260000A431A601968044A0A401A607047C04647
:10327000080200500C000050FFFFCFFF072318404A
:103280001B4B80001B5810B59F461A4804681A4B08
:103290000904234019430123016081681A400F3358
:1032A000120199430A43826010BD1448090603685D
:1032B0001B021B0A0B430360012381681A401F3362
:1032C000520199430A438260EEE70C48DEE7094861
:1032D000090603681B021B0A194301231A40530104
:1032E00020220160816891430A001A438260DBE773
:1032F000288D000000001440FFFF00FF0000044084
:1033000007230340043BDAB210B5032A20D938243E
:10331000C20014400122A240204B00241B689343AA
:10332000002924D11D4A23431360C3060FD510384A
:10333000C0B207280BD81A4B80001B589F46194A69
:103340001168194B0B40802109030B43136010BD1A
:103350000124164ADB0012689C4013000022A3439C
:10336000002900D022001343104A1360DDE7140047
:10337000D8E70F490A680F4B1340082213430B602C
:10338000E5E70849F6E70C4ADAE70B49F2E70B4AAA
:10339000D6E70A49EEE7064AD2E7C04608000440ED
:1033A000488D0000500014400F0007000800144032
:1033B0005400144007000F00540004405000044023
:1033C000F0B556464D4644465F46F0B40724D44A0D
:1033D0000440A300D35883B006000D009F46D14B94
:1033E000DB699B069B0F002B0ED0022B00D16CE1FA
:1033F000CD4B9A46172E1CD8CC4AB300D3589F46C3
:10340000C84B5B699B0FF0D1C94B9A46F2E7C54B9D
:103410005B699B009B0FE6E7C24BDB691B069B0FBA
:10342000E1E7C448EA6803681104C34A13400B4348
:103430000360271FFBB2032B00D8BFE03821F20046
:103440000A40033237399140BC4B28781B680A0088
:103450008B430021002800D0C0E0B84A0B43136022
:103460006968002906D1072C00D9DDE0B44AA30021
:10347000D3589F46504604F0A5FF802383465B0542
:1034800000209B4500D992E0AE4B9B4500D8A7E0B9
:103490005B46190C8BB25846994604F093FF802383
:1034A0005B02984203D94B4601339BB29946802375
:1034B000C8465B00994500D895E05A465B46110E18
:1034C0001B0ACAB218000193904604F07BFF8023C8
:1034D0005B02984200D98FE1002301200200591CB1
:1034E0009A40CBB24245F9DD0122013B9A401300DC
:1034F000D2B291460020102A59D8FF221A4011005A
:103500000198904604F05EFF83B200040193030C1F
:103510009B4653464146180A04F054FF594604F0AE
:1035200051FF8046072C00D981E1874AA300D35878
:103530009F468649FF200B68EA78834313430B605C
:10354000AB68687864215843984604F03BFFFBB2AF
:103550000138032B00D89FE01C23B6001E40153B0A
:103560001A00B2407A490F689743AA781340B340D3
:1035700042463B430B6063001C19764BA400E318E2
:10358000013A1A60744B9C4664442060AB78012475
:10359000032B01D8714AD45CE9785046013104F01C
:1035A00011FF210004F00EFF414604F00BFF03B0B1
:1035B0003CBC90469946A246AB46F0BD0122F900BC
:1035C00003318A40664B28781B680021934300280A
:1035D00000D01100624A0B43136041E711003CE741
:1035E0000223984699464146584604F0EBFE83B2C2
:1035F00000040193030C9B464146504604F0E2FE52
:10360000594604F0DFFE8046072C00D981E0554A78
:10361000A300D3589F4654490868EA78534B1202D6
:10362000034013430B608BE74F4983E7414A11681E
:10363000414B0B40E9680B431360FAE64C48F1E656
:103640004B4AF4E74B48EDE64A4AF0E74A48E9E6D8
:10365000494AECE70122F1001E398A40404BE868F4
:103660001B6800219343002800D011003C4A0B4303
:103670001360DEE60122F10002318A402F4BE86838
:103680001B6800219343002800D011002B4A0B43F4
:103690001360CEE62D49BFE707231A00BE00B240F3
:1036A000364C21689143AA781340B34042460B43FD
:1036B00023607B00DF19324BBF00FB18013A1A6010
:1036C000304B9C466744386060E72F4B1B689A4636
:1036D00090E601224B469146013BDBB21B49FF209D
:1036E0000A68824313430B600BE001224B4691466C
:1036F000013BDBB21C491A0208681C4B0340134310
:103700000B604B46102B00D988E0204A9B00D35811
:103710009F464B460122013BDBB291461249DEE750
:10372000688D00000002005000805101888D00006B
:10373000001BB700540014400F000F0008000440A5
:10374000E88D0000FFFF0100088E0000000014401B
:10375000040004400C00044010000440AC8E000043
:1037600008001440288E000000000440FF00FFFF06
:103770005000144054000440500004400400144021
:103780000C00144010001440F8000020488E000087
:1037900000239946F30652D5A8686421431E9BB2C4
:1037A0009A466B78584304F00DFEFBB2013880B2A4
:1037B000032B54D91C21B6000E401539B140334AB1
:1037C00013688B434946B1400B4313605246630074
:1037D0001C192F4BA400E3181A602E4B9C4664441E
:1037E00020604046E3E601239946D3E70323994648
:1037F000D0E702239946CDE743460133DBB2984632
:103800006AE601234A469946013AD2B22249234B3D
:1038100008681202034013430B6072E74A4607230D
:103820001A409146B6E7FF2358E7FF2362E7FF23DC
:103830001B4954E7FF22E9E704239946AAE7019BC5
:103840006878013B9BB29A465B464343642118006B
:1038500004F042FEFBB2013880B2032BAAD8072243
:10386000BC00A2400F490B6893434A46A240134351
:1038700052460B607B00DF190B4BBF00FB181A6030
:103880000A4B9C4667443860404690E6040004407A
:103890000C0004401000044000001440FF00FFFF33
:1038A00000000440040014400C00144010001440B8
:1038B00000290BD0C3061ED5430726D50123143893
:1038C000834022498A6F13438B6713E0C30609D5EF
:1038D00043072AD50122143882401C498B6F934339
:1038E0008B6707E0430729D40122824018490B68FF
:1038F00093430B607047430710D50123043883407E
:1039000014490A6813430B60F4E707231840063B89
:10391000834011498A6F13438B67EBE70123834090
:103920000B490A6813430B60E4E707221040063A8C
:10393000824009498B6F93438B67DBE70122043890
:10394000824004490B6893430B60D3E700001440A6
:103950007C0004407C001440000004400723184011
:10396000154B80001B5810B59F4603231348194080
:10397000C2692D3309019A431143C16110BD0F4A39
:10398000890753699B009B080B435361F6E70323A8
:103990000A48194044690B072100094A114019439C
:1039A0004161EBE70320054A0140D369BD3089013D
:1039B00083431943D161E1E78C8E0000000200507F
:1039C000FFFFFFCFA02280230021D2055B00D15052
:1039D000D358DB0701D4002070470148FCE7C046FC
:1039E0000296FFFFA0220123D20591680B4393604A
:1039F0007047C046A022102310B5D20591690B4331
:103A00009361034B1B68002B00D0984710BDC04644
:103A10002802002023280FD0222817D0104A13682C
:103A2000002904D1012181408B431360704701219B
:103A300081400B431360F9E70A4A2238536801407A
:103A40000730C900834319435160EFE7054A213825
:103A50005368014003308900834319435160E5E70F
:103A6000080200500002005010B50B2868D8354BF2
:103A700080001B589F46032333481940C26909013F
:103A80002D339A431143C161002010BD03232E48FA
:103A90001940C2698901BD33F3E703202A4A014076
:103AA00053698343194351610020EEE703232648FD
:103AB00019404269093389009A431143416100204A
:103AC000E3E70723204819404469204A0B022100FC
:103AD0001140194341610020D7E707231A481940D4
:103AE00044690B031A4AF2E707231748194044694F
:103AF0000B04184AEBE707231348194044690B05E8
:103B0000154AE4E703231048194044690B06134A99
:103B1000DDE703230C48194044690B07104AD6E738
:103B2000094A8907536900209B009B080B43536196
:103B3000ABE7032304481940C26989000933A0E7B1
:103B40000848A2E7B08E000000020050FFF8FFFF17
:103B5000FF8FFFFFFFFFF8FFFFFF8FFFFFFFFFFC5F
:103B6000FFFFFFCF0496FFFF402310B5044A116802
:103B70000B431360034B5B68002B00D0984710BDCC
:103B8000000200502802002000487047001BB700C8
:103B900030B585B06A46154B6D4613CB13C21B6812
:103BA0001360134B1B6A1B0318D4114B114A196A7B
:103BB000C90318D4186A196A1C6AC005C00D8904A3
:103BC0002404C90EA40F023002315043A40004F0B3
:103BD000F9FB295904F0F6FB05B030BD044B064A49
:103BE000196AC903E6D50020F6E7C046E08E00005A
:103BF00000020050001BB7000080510110B50F4AB1
:103C000013695B0712D013695B075B0F022B11D09E
:103C100013695B075B0F032B0AD00948074B9969AF
:103C20000907090F013104F0CDFB10BD0548F5E788
:103C30000548F3E7FFF7ACFFF0E7C046000200508D
:103C400000805101001BB70010270000F0B544466A
:103C50005F4656464D460422F0B48024C94BCA48FC
:103C6000D96802621A68E404224380241A601A6840
:103C7000E40522431A600022C44B1A80C44A136828
:103C80009B0603D4C34B1C78092C54D90020C24B8B
:103C90001880642949D9C14B02301C68204234D0B5
:103CA0001C680E30204200D086E01868800600D4E0
:103CB00092E004201C68204200D1C8E01C688443C4
:103CC0001C6080241868A0431860B548814202D85F
:103CD00019680C431C6080201968084200D0C5E0B8
:103CE000B049B14CB14E0A783078D2B2C0B2A054CB
:103CF00020201A6882431A600A780132D2B20A7010
:103D00000A78102A11D9AA4A08E0A54A914257D93F
:103D1000A74A1178122900D979E0A2491C68A54860
:103D200020401860002313700B703CBC90469946ED
:103D3000A246AB46F0BD994C2568AD001FD49E4D00
:103D40002D78002D1BD025686D059FD42468640252
:103D50009CD41C780134E4B21C701B780A2B95D1DA
:103D60000525964C76332370954C2570954CA568A7
:103D70002B43A36040248368A343836086E7924873
:103D80000078C0B2002821D018780130C0B2187075
:103D90001B780A2B00D079E7052488487633037016
:103DA00087480470874884682343402483607648AA
:103DB0008368A343836069E71A6882431A60B4E7A3
:103DC0007B4A13780133DBB21370AEE707247C4BD8
:103DD0001C707A4B187059E7744802785200D2B2BE
:103DE00002706F4A91422DD971490A780132D2B2DC
:103DF0000A700A78072A05D92022186802431A6037
:103E000000220A70102219680A431A608DE71968A7
:103E1000490702D51968084318600421186801434E
:103E200019601968890700D47FE7FF20196881436A
:103E300019600A2118680143196000231370594A58
:103E4000137072E702780132D2B20270CCE71A68BE
:103E50001043186040201A6882431A60504A914209
:103E600000D962E71A68104318605EE70425574CD2
:103E7000A1686940A1604B490E78012E00D842E745
:103E8000534EB3467679B44601266746B2463E4263
:103E900066D0504FBC463F6AB9464F4FB8464F4672
:103EA00046463740664637624C4E3550604655466A
:103EB000006A8026A84365462862494DF6052868B1
:103EC000304328600025474805700820A668304325
:103ED000A06040202C4CA66830438026A06010686B
:103EE00076023043106040482F4C05702078FF2840
:103EF00039D02E4E0A783078D2B2C0B2A0540A78A7
:103F000000200022A55C013268400D78D2B29542B3
:103F1000F8D2002800D0F6E63F252278AA43802A6E
:103F20006CD01A68314D324F2A431A600A783870C3
:103F3000002A00D1A0E000222E4DA05CC0B2A854FF
:103F400008780132D2B29042F7D83A700A783078C5
:103F5000D2B2C0B2A854F2201A6882431A60C2E6F4
:103F60000A78114CC5E760780335A843FC28C0D116
:103F7000214DA8680643AE60802510686D01284376
:103F80001060B6E720001140C040005080050020BE
:103F90009007002082050020840500207C05002079
:103FA000FF0700004A040020BC0200201E0300207E
:103FB0008907002000FFFEFF1D030020860500206A
:103FC000AE020020004000507405002080400050E8
:103FD000F002002000000E40FFF7FFFF00E100E0CC
:103FE00000001140B80200204C050020010008002C
:103FF0003002002008030020000200501A68D2009E
:104000000CD522783348D2B2027062783248D2B2EC
:10401000027080201A68800002431A605A46527962
:10402000D20604D55A46D07A2278904226D05A46F3
:104030005279920600D466E65A46557B2078274A84
:10404000854200D06AE658460125867B6078A84301
:10405000B04200D062E6607828401DD0002420489D
:1040600004702048803404701C681F4820400524D8
:1040700018601E48047051E61D4D67E75A46107BD4
:1040800062789042D3D180201A6840040243002015
:104090001A60184A1080CAE70227174CA6683E43E8
:1040A000A660A668FF19BE43A660144E7C37B468AC
:1040B000BC43B460124E403FB4683C43B460094C0A
:1040C000207081241868A4052043186007480570F3
:1040D00024E6C0462F0300208C070020890700201B
:1040E0008205002086050020FFFFBFDFAE02002012
:1040F00008030020960700200041005000400050B7
:10410000C04000500822304BF0B51A622F4A304BA5
:1041100011680B402F4913600B685B0349D580235E
:1041200008689B02184245D07F2408682A4B034048
:104130002A480B600378234003708020052513680C
:10414000C00403431360264B264F1C78E4B2601C66
:10415000C0B21870244805551C78E4B2651CEDB255
:104160001D70042505551C78E4B2651CEDB21D7068
:10417000002505551C78E4B2651CEDB21D703D7834
:10418000EDB26E1CF6B23E7005551C78E4B2651CAB
:10419000EDB21D70872505551C78E4B2651CEDB2A3
:1041A0001D700B689B03DB0F035511680F4B0B4011
:1041B0001360F0BD086803430B6080230748047850
:1041C00023430370B9E7C046C04000507C0500207F
:1041D000FFFFDFFF90070020FFFFFDFFAE02002082
:1041E000EC0200204D0500204C040020FFFFFFFBE7
:1041F000F0B54F464646AC4AC0B4138801339BB273
:104200001380AA4A138801339BB21380A84B9946A6
:104210001B88002B05D04B464A461B88013B9BB2AE
:104220001380A44A13780133DBB21370A24B1A68CF
:10423000002A02D01A68013A1A60A04B1A88002A94
:104240000CD01A88013A92B21A801B88002B05D133
:1042500000229B48C25401330A2BFBD1994B1A68A8
:10426000D20100D4B6E098480278802A00D117E243
:104270000024964A14801488954A944200D8A9E0F4
:104280008022944D944FAC689443AC604024934D8D
:10429000AE683443AC600426002581243E7005706E
:1042A0001868A405204318608D488E4C07683C4070
:1042B000046090248C4FB9680C43BC6080278B4C01
:1042C000BF01A750A6508A4C8A4A25701588002D38
:1042D00000D086E0884D2A88013292B22A80874A2F
:1042E0001588002D03D01588013DADB21580844A94
:1042F0001588002D00D082E0824D2A88002A08D03F
:104300002A88013A92B22A802A8892B2002A00D1E1
:1043100086E17D4D2A78D2B2002A00D17FE0FA27CB
:104320007A4EBF007288BA4200D876E100227280CD
:104330002A78013AD2B22A70754D2A8892B2561C58
:10434000B6B22E80C82A00D16DE12A88C72A03D8C8
:104350001A68520400D540E16E4A1668002E06D055
:104360001668013E16601268002A00D132E16A4FD9
:10437000BA79002A0CD0654EB28894460132B280D8
:10438000BA799100884642445200944500D17FE1B9
:10439000624E3288013292B232802278D2B2002A42
:1043A0005CD05F4A176801371760C8271168BF00E3
:1043B000B94200D9C4E08022016892020A4040D08C
:1043C000FF2233881340802B00D149E10CBC90467A
:1043D0009946F0BD474A42481588454C002D00D10A
:1043E00078E71588ADB26E1EB6B21680012D00D0EA
:1043F00070E720263C4DAA68B243AA606AE7158898
:10440000484E013DADB215803E4D2E801288002AE7
:1044100000D072E740260268B24302606DE7424D69
:104420002D78002D00D187E7274D2D786DB2002D16
:1044300000DA81E71E683D4D35401D603C4D2A7015
:104440007AE73C490888002824D1234F3B78DBB227
:10445000092BBBD8384A9B00D3589F467979490726
:10446000A9D5364F398889B24C1CA4B23C80FA24B5
:10447000A400A1429FD910213A801B4A146921420D
:1044800000D138E194688C43802194609468214382
:10449000916090E70888012800D107E10E4F0B8852
:1044A000013B9BB20B80D1E7300300208A0700203C
:1044B000E402002059050020E0020020440300200F
:1044C000200300207C0500208605002096070020A0
:1044D000B036000000400050AE020020C040005046
:1044E00090070020FFFFFBFF8040005000E100E04C
:1044F000A4070020BA0200204E050020A2070020D9
:10450000A00200202C0300207805002030020020AB
:104510008405002054050020F002002076050020CC
:104520009C070020881300001D030020FFFFBFFF31
:1045300082050020B0020020F08E000080050020DF
:1045400000210F271160B94A8C4612683A40B84FD3
:1045500040323A70B74A21701170B74AB74C1170A7
:104560009022A7683A43A26001248027B44A1470BD
:10457000B44CA268BA43A2604022B34CA7683A4345
:10458000A260B24FB24C397021801F68B14C4946CD
:104590003C401C600424B04F00223C60FA27BF005E
:1045A0000F800627AD490F70AD490A701F68AD49ED
:1045B00039401960AC490A70AC490A70AC4A91683C
:1045C0000C43022194609468214391606146A94A9A
:1045D0001160F0E6A84E3260C9E600264021A04AEC
:1045E000984F1670BA6880363243BA60964FBA68F0
:1045F0008A43BA60994A954F167005223A701E6830
:10460000984A324080261A600268F60432430260FB
:104610001E689A4A32401A609EE6013272808BE62A
:10462000974D2A7075E68027864EB268BA43B2600D
:104630004022854EB7683A43B2600022884E834FCD
:104640003270834E32801E68824A32401A600622DF
:10465000824E32702678002E18D100223A7074E60D
:10466000884A9379012B00D1D2E0002B00D1C3E01E
:10467000022B48D0002302219371834B9A688A430E
:1046800004219A609A688A439A609FE63A705CE6D1
:1046900080211A6809040A431A600022B28077E672
:1046A0007A4A14880134A4B21480E4E51C6869488D
:1046B000664F20401860694B1B785BB2002B00DA14
:1046C000B1E03A70EBE6FA232A889B009A4200D0C8
:1046D0007CE600236B4A2B80137A591C1172DB078E
:1046E0004CD40422684B99680A439A600222996864
:1046F0000A439A606AE69468214380249160916835
:10470000A143916057E660498868034304208B60A9
:104710008B6883438B600323937157E68022338831
:104720005200DB05DB0D934200D04FE6554BDA79A2
:10473000511CD971052A00D948E6554992008A587A
:10474000974633889B0607D502224F4B99680A4348
:1047500096E733881B06F7D402214B4A93688B43B4
:10476000936033E633885B0608D50423464A916894
:104770000B4393602AE633885B06B2D40421424B94
:104780009A688A439A609A6802398A439A601DE659
:10479000FA232A889B009A4200D017E600233A4A5F
:1047A0002B80916804334B4093600FE60422364B14
:1047B00099680A4302219A609A688A439A6005E6DA
:1047C000802233885200DB05DB0D934200D0FDE5EB
:1047D0002C4BDA79511CD971052A00D9F6E52D49FF
:1047E00092008A5897460022DA71EFE50223264AA2
:1047F00091680B439360E9E50421234B98680143DA
:104800000220996099688143996001239371DDE5E5
:1048100002201D4B99680143996004219C68214343
:1048200099609071D2E505233B7038E6B402002010
:104830004904002088070020A50700208040005080
:104840001D03002000400050C0400050AE02002078
:10485000B0020020FFFFFFBF00E100E0860500205E
:1048600082050020FFFFBFDFEC0200209807002038
:1048700000001540CC02002070420050FFBFFFFF37
:10488000580500203002002000410050960700200B
:10489000188F0000308F0000F0B55F4656464D4639
:1048A00044468021E04AF0B4136849020B43DF48D4
:1048B0001360037885B0DBB2591CC9B20170042BB8
:1048C0000ED8DB499B00CB589F460821D94A9368F4
:1048D0008B4393608021D84AC90513680B4313604A
:1048E00005B03CBC90469946A246AB46F0BD802040
:1048F000D249C0040B78013BDBB20B70D0490B6886
:10490000034380200B600B68C0050343CD480B6058
:10491000CB688342FCD900200121CB4B1870CB4BD4
:104920001870CB4B1C6A2143CA4C1962A568CA494E
:104930002940A1604024C94DA968A143A96004256C
:10494000C7490D608025196A2D0129431962C54B9D
:1049500059790C4230D1C44910231068034205D064
:104960000324C24804601068984310601068C04B6C
:104970000340136000230022CA540133082BFBD1EB
:10498000AEE78020AC49C0050B68034308200B60EC
:10499000A8498B6883438B6013685B0305D580212E
:1049A000AC4A490293680B4393600222B14B996869
:1049B0000A439A601B6893E7AB490C78002CCBD074
:1049C0000C780F2CC8D90C78EF2CC5D80C78AA4DD0
:1049D0000F3CE4B22C5DE4B2402C01D100F038FC75
:1049E000A608F5B2072D01D100F0ACFC00D9FDE01E
:1049F000002DB1D14B780E2BAED900209F4B186003
:104A00004B789D480F3BC35CDBB20293402BA3D095
:104A10009B4803785BB2002B01DA00F08BFD8378B2
:104A2000DBB2C3704378DBB283700378DBB24370D0
:104A3000002301930F258378AB43E02B02D00023A2
:104A40008370C3708F4B00259C4663465B5D984620
:104A5000435D984501D000F061FD0135052DF4D18D
:104A6000894D2B7B5E1C2E73012B00D074E71368DD
:104A70005B0300D4B5E0854B80259C461B68ED04A4
:104A80002B43654609272B60814BB9461D784E465E
:104A9000EDB2A84647460135EDB21D707D4DA4012B
:104AA000EE556F461E78E4B2FE73FE7B0127B046DA
:104AB00047443E1C6F46FE73FE7B1E700826B146BF
:104AC00046464F46AF556F461E78FE73FE7B012764
:104AD000B04647443E1C6F46FE73FE7B1E700026A8
:104AE000B14646464F46AF556F461E78FE73FE7B75
:104AF0000127B04647443E1C6F46FE73FE7B1E7086
:104B0000654EB3463678FE73FE7B0127B1464F44AF
:104B10003E1C6F46FE73FE7BB2465E4657463770BC
:104B200046464F46AF556F461E78FE73FE7B012703
:104B3000B04647443E1C6F46FE73FE7B1E70A526A2
:104B4000B14646464F46AF556F461E78FE73FE7B14
:104B50000127B04647443E1C6F46FE73FE7B1E7025
:104B60004678FE73FE7BB14646464F46AF556F46CC
:104B70001E78FE73FE7B0127B04647443E1C6F46FD
:104B8000FE73FE7B3F791E704646AF551E78F6B227
:104B9000B146771C6E463771FFB21F70C778377108
:104BA00037794E46AF551E78F6B2771CB1466E4641
:104BB000377137794E461F7080788046032047460C
:104BC0003840A8551878C0B2461CF6B21E702300B3
:104BD000029C23432B5463461868304B03406046C5
:104BE0000360C8202E4B80001880B5E60E3E012ED3
:104BF00000D9B1E61368DB0400D4ADE600201F4BFA
:104C0000A4011860E3B201934B781B480F3BC65CCC
:104C10001B48F6B243780533DBB2042B00D99BE680
:104C2000204D9B00EB589F4690070020B8020020C3
:104C3000488F000080400050000011402E030020EB
:104C40002000114061020000890700204A04002072
:104C500000000E4000020050FFFFFEFFC040005069
:104C600000E100E0F0020020A40200205405002032
:104C7000FFEFFFFF000005400000002070420050E1
:104C8000BC02002020030020300200207C05002010
:104C9000EC0200204C0400204D050020FFFFFFFB2C
:104CA000440300205C8F00001368402E01D100F007
:104CB00045FD5B0300D44FE6C84B80209C461B6833
:104CC000C004034360460A276C460360C44B1D784A
:104CD000EDB2681CC0B21870C24847551D78EDB2DD
:104CE0006F1C2772FFB21F70092747551D78EDB260
:104CF0006F1C2772FFB21F70002747551D78ECB25A
:104D00006D46671C2F72FFB21F70B74FBA463F78CF
:104D1000FFB2B846012747442F72FFB2B946574643
:104D20004D463D70454605556C461D78EDB26F1CED
:104D30002772FFB21F70B32747551D78EDB26F1C65
:104D40002772FFB21F70FF2747551D78EDB26F1C09
:104D50002772019CFFB234431F7044558C78A34DD9
:104D60000F3C2C5DCD78A14E0F3D755DA401E4B2E2
:104D70002C431D78EDB26E1CF6B21E7044550C79B2
:104D80009A4D0F3C2D5D4C79984E0F3C345DAD0033
:104D9000E4B22609EDB23543A9466D461E782401DA
:104DA000F6B2771C2F712F794D461F7085558D797E
:104DB0008E4E0F3D755DE4B2EDB2AE083443A146B0
:104DC0006C461E78AD01F6B2771C277127794C46E8
:104DD0001F708455CC79854E0F3C345D2C431D7873
:104DE000E4B2EDB26E1CF6B21E704455634618680C
:104DF0007F4B034060460360AEE5402E00D1ABE53B
:104E000013685B0300D4A7E5744B80259C46644679
:104E10001B68ED042B432360714B1D78ECB2A04658
:104E2000651C0A24A14644464F46EDB21D706D4DE7
:104E30002F556F461C783C723C7A0127A0464744A8
:104E40003C1C6F463C723C7A1C700924A1464446C7
:104E50004F462F556F461C783C723C7A0127A0467E
:104E600047443C1C6F463C723C7A1C700024A146AF
:104E700044464F462F556F461C783C723C7A0127BA
:104E8000A04647443C1C6F463C723C7A1C70564C12
:104E9000A34624783C723C7A0127A1464F443C1C2F
:104EA0006F463C723C7AA2465C46574627704446A1
:104EB0004F462F556F461C783C723C7A0127A0461E
:104EC00047443C1C6F463C723C7A1C70B524A1469A
:104ED00044464F462F556F461C783C723C7A01275A
:104EE000A04647443C1C6F463C723C7A1C70FF2431
:104EF000A14644464F462F556F461C783C723C7A7B
:104F00000127A04647443C1C6F463C723C7A374F11
:104F10001C70019C34434646AC558C78334E0F3C94
:104F2000345DCE78A4010F3EBE5DE4B23443A146A9
:104F30006C461E78F6B2771C277127794C461F7095
:104F4000AC550C79294E0F3C365D4C79274F0F3C00
:104F50003C5DB600E4B2A24627096C46F6B2374380
:104F6000B8461E78F6B2771C2771277954461F7011
:104F70004746AF558E791D4F0F3EBE5D2401F6B2F8
:104F8000B046E4B2B6083443A2466C461E78F6B288
:104F9000771C2771277954461F70AC55CC79134E76
:104FA0000F3C365D4446A40134431E78E4B2F6B2A9
:104FB000771CFFB21F70AC551C78E4B2661CF6B2C9
:104FC0001E70C679F6B22E551C78E4B2661CF6B295
:104FD0001E70C023007A03432B5507E77C05002091
:104FE000EC0200204C0400204D05002000000020B1
:104FF000FFFFFFFB1368402E01D100F008FC5B03AC
:1050000000D4A9E4C94B80259C461B68ED042B43C2
:1050100065460F272B60C64BB9461D784C46EDB24E
:10502000A84647460135EDB21D70C24DEC556F469E
:105030001C783C723C7A0127A04647443C1C6F46D2
:105040003C723C7A1C700424A14644464F462F55BE
:105050006F461C783C723C7A0127A04647443C1CB2
:105060006F463C723C7A1C700024A14644464F4671
:105070002F556F461C783C723C7A0127A046474466
:105080003C1C6F463C723C7A1C70AB4CA3462478A7
:105090003C723C7A0127A1464F443C1C6F463C724F
:1050A0003C7AA2465C465746277044464F462F55E9
:1050B0006F461C783C723C7A0127A04647443C1C52
:1050C0006F463C723C7A1C70B424A14644464F465D
:1050D0002F556F461C783C723C7A0127A046474406
:1050E0003C1C6F463C723C7A1C70FF24A14644462F
:1050F0004F462F556F461C783C723C7A0127A046DC
:1051000047443C1C6F463C723C7A1C7084783C726D
:105110003C7AA14644464F462F556F461C783C7258
:105120003C7A0127A04647443C1C6F463C723C7ABF
:105130001C70C4783C723C7AA14644464F462F55B9
:105140006F461C783C723C7A0127A04647443C1CC1
:105150006F463C723C7A1C7004793C723C7AA146E2
:1051600044464F462F556F461C783C723C7A0127C7
:10517000A04647443C1C6F463C723C7A1C70447904
:105180003C723C7AA14644464F462F556F461C78E8
:105190003C723C7A0127A04647443C1C6F463C7257
:1051A0003C7A1C7044468079C0B228551878C0B249
:1051B000441C3C723C7A1C70019C34432C5488780B
:1051C0005E4C0F38205CCC785C4E0F3C345D800127
:1051D000C0B220431C78E4B2661CF6B21E7028559B
:1051E0000879564C0F38245C4879544E0F38305C9F
:1051F000A400C0B20609E4B23443A1466C461E784E
:105200000001F6B2771C277127794C461F70AC5508
:105210008C794A4E0F3C345DC0B2E4B2A6083043EC
:10522000814668461E78A401F6B2771C077107799B
:1052300048461F70A855C879404E0F38305C20434F
:105240001C78C0B2E4B2661CF6B21E702855CDE5DB
:105250001368DB0401D4FFF77FFB13685B0301D401
:10526000FFF77AFB80240A27304DE4042B682343A0
:105270002B602F4B1E78F6B2741CE4B21C702D4CC0
:10528000A7551E78F6B2771CFFB21F700927A755E5
:105290001E78F6B2771CFFB21F70A0551E78F6B2CA
:1052A000771CFFB21F70244FB146B8463F78FEB25C
:1052B0006F46B24601363E713E79B4464646674671
:1052C00037704E465746A7551E78F6B2771CFFB288
:1052D0001F70B327A7551E78F6B2771CFFB21F7058
:1052E000FF27A7551E78F6B2771CFFB21F70A05596
:1052F0001E78F6B2771CFFB21F70A0551E78F6B26A
:10530000771CFFB21F70A0551E78F6B2771CFFB253
:105310001F70A0551E78F6B2771CFFB21F70A05503
:105320002868074B03402B60FFF716FB7C05002025
:10533000EC0200204C0400204D050020000000205D
:10534000FFFFFFFB4D780E2D01D8FFF705FBF04D59
:10535000286088780F2808D9C878EF2805D8887879
:10536000EC4C0F38C0B2245CE4B2012C00D1C6E191
:10537000002C00D1E4E0072C01D0FFF7EDFA08780B
:10538000E44C0F38C0B2255CE8B2019048780F3881
:10539000C0B2275CF8B20290DF48047864B2002CF7
:1053A00000DAB0E18478E4B2C4704478E4B2847086
:1053B0000478E4B244700024A4469C7C002C01D103
:1053C000FFF7CAFAD54C26889B7C9846642345464D
:1053D0006B439E4201DCFFF7BFFA0023238099460E
:1053E00013685B0301D4FFF7B7FA80240925CC4E7C
:1053F000E4043368AA4623433360CA4B57461C78FB
:10540000E4B2A04645460134E4B21C70C64C675570
:105410006F461D78FD73FD7BA84601254544FD734D
:10542000FD7B1D700825AA464546574667556F46C1
:105430001D78FD73FD7BA84601254544FD73FD7B6A
:105440004F461D70454667556F461D78FD73FD7BC1
:10545000A84601254544FD73FD7B1D70B34DAB4649
:105460002D78FD73FD7BA94601254D44FD73FD7B21
:10547000AA465D4657462F7045464F4667556F46CC
:105480001D78FD73FD7BA84601254544FD73FD7B1A
:105490001D70AA25A94645464F4667556F461D789B
:1054A000FD73FD7BA84601254544FD73FD7B1D7002
:1054B000FF25A94645464F4667556F461D78FD7343
:1054C000FD7BA84601254544FD73FD7B1D704546C7
:1054D0004078C0B260551878C0B2451CFD73FD7BA2
:1054E0001D70654625541878C0B2451CFD73FD7BC0
:1054F0001D70012525541878C0B2451CFD73FD7B35
:105500001D70029D019BAC469B016344DBB223549A
:105510003068874B03403360FFF71EFA0023854C49
:1055200023736546C45CE4B2EC540133052BF8D117
:10553000FFF712FA3F2306781E400196FFF77AFA2A
:10554000002084460878734C0F38C0B2255C487838
:10555000EDB20F38C0B2245C6F48E4B2067876B280
:10556000002E00DAC9E08678F6B2C6704678F6B248
:1055700086700678F6B246700026077801967FB2EC
:10558000B74203DA07783F363E40019617687E033C
:1055900001D4FFF7E1F9674FAD0164197D89E4B2E9
:1055A00064196444A4B264087C815D79A3466DB239
:1055B000002D01DBFFF7D0F95F4D2F88DB7C9C4687
:1055C0000A23664673439F4201DCFFF7C5F90023B7
:1055D0002B8080250826524F98463B68ED042B43CC
:1055E0003B60504BB1461D784C46EDB2AC4666462A
:1055F0000135EDB21D704C4DAC556E461C783472C1
:10560000347A0126A4466644341C6E463472347AD9
:105610001C700724A14664464E462E556E461C78E3
:105620003472347A0126A4466644341C6E463472C1
:10563000347A46461C7064462E556E461C78347289
:10564000347A0126A4466644341C6E463472347A99
:105650001C70364CA24624783472347A0126A04657
:105660004644341C6E463472347AA14654464E4643
:105670002670644646462E556E461C783472347A3F
:105680000126A4466644341C6E463472347A1C707B
:10569000A624A046644646462E556E461C783472B3
:1056A000347A0126A4466644341C6E463472347A39
:1056B0001C7064464078C0B228551878C0B2441CAB
:1056C0003472347A1C7034792C5418785C46C0B229
:1056D000461CF6B21E706E46347136792E54187818
:1056E000C0B2461CF6B21E705B461C0A2C543868C9
:1056F0000F4B03403B60FFF72FF906783CE7802013
:10570000400084461EE73F2406782640B44654E60F
:105710007042005000000020BC0200208A070020D8
:105720007C050020EC0200204C0400204D050020E8
:10573000FFFFFFFB30020020300300205B0301D499
:10574000FFF70AF980200A26834DC0042B68034323
:105750002B60824B1C78E4B2601CC0B21870804889
:1057600006551C78E4B2661CF6B21E700926065572
:105770001E78F6B2741CE4B21C70002484551E78A6
:10578000F6B2771CFFB21F70764FB146B8463F782D
:10579000FEB26F46B24601363E713E79B446464689
:1057A000674637704E46574687551E78F6B2771CC7
:1057B000FFB21F70B32787551E78F6B2771CFFB271
:1057C0001F70FF2787551E78F6B2771CFFB21F7037
:1057D00084551E78F6B2771CFFB21F7084551E7870
:1057E000F6B2771CFFB21F7084551E78F6B2771C94
:1057F000FFB21F7084551E78F6B2771CFFB21F707F
:1058000084552868584B03402B60FFF7A5F85B03CD
:1058100001D4FFF7A1F8504B80249A461B68E4049A
:10582000234354460F2723604C4B1D78EDB26C1C6C
:10583000E4B21C704A4C67551D78EDB26F1CFFB284
:105840001F70042767551F78FFB27D1CEDB21D70D5
:105850000025E5556D461F78FFB2BC460137FFB203
:105860001F70404FB9463F78FEB2B34601362E71E5
:10587000F6B2B0464E464746377066465F46A75575
:105880001F78FFB27E1C2E71F6B21E70B426E6554C
:105890001F78FFB27E1C2E71F6B21E70FF26E655F1
:1058A0001F78FFB27E1C2E71F6B21E7086782E71A4
:1058B000F6B2E6551F78FFB27E1C2E71F6B21E704E
:1058C000C6782E71F6B2E6551F78FFB27E1C2E7197
:1058D000F6B21E7006792E71F6B2E6551F78FFB249
:1058E0007E1C2E71F6B21E7046792E71F6B2E65508
:1058F0001F78FFB27E1C2E712E7900251E708079D4
:10590000C0B2E0551878C0B2471CFFB21F702554D2
:1059100000251878C0B2471CFFB21F70255400251F
:105920001878C0B2471CFFB21F70255400251878A4
:10593000C0B2471CFFB21F7025541878C0B2471C74
:10594000FFB21F700023235453461868064B0340D0
:1059500050460360FFF700F87C050020EC020020B1
:105960004C0400204D050020FFFFFFFBF0B583B085
:105970006A46224BD41D1B680025DBB2237000232E
:105980000026002101201E4F2278BB7308331042ED
:1059900003D00131C9B20E000125013BDBB2520830
:1059A000002BF4D1002D27D108237A73FB7304292F
:1059B00001D003B0F0BD134B1A68520314D4124A3D
:1059C00012481378DBB2591CC9B211702178C9B2E0
:1059D000C1541378092BECD9002313700C4A0D4BDA
:1059E00091680B409360E4E70B4A03391160102281
:1059F00019680A431A60E2E7BE73D5E70000054064
:105A000030020020900700204C050020A402002056
:105A100000020050FFFFFEFF70420050F0B55746F5
:105A20004E464546E0B482B06946CE4A1368DBB2C2
:105A3000CB7193691B07D80F002B36DBCA4A13685A
:105A4000002B00DA2EE1C949C9480B78013B5B0005
:105A50001C5A80235B009C4200D172E0C14B9A69C2
:105A6000120403D5022299680A439A60BD4B9A69D1
:105A7000D20707D5012299690A439A6102229968DF
:105A80000A439A60B74B9A6992060AD50223B54A2F
:105A900091680B43936002B01CBC90469946A246A5
:105AA000F0BD9B69DB06F1D4F5E7082593692B432C
:105AB0009361CB7940210B4057D169467F24C97946
:105AC000214000D182E1AB490978C9B2022900D155
:105AD00098E10329C2D169461F24A748C9790078F3
:105AE00021408142D7D1A54C23601023D1680B43BC
:105AF000D3602023D1680B43D360D3682B43D3609A
:105B000013009A69974FD200FBD59D4B1A688023EA
:105B1000DB04134000D0D6E19A4E9B4A30781178CE
:105B2000884200D106E233789849DBB2CD5C8846E2
:105B3000EDB22B1F3B2B00D8C8E11378DBB23370DA
:105B4000A9E70B78DBB25C1CE4B20C706946C9793A
:105B50005B0019528021136809060B431360814BC7
:105B60009A69120400D481E77CE76B467F22DB79D7
:105B700013407D2B00D141E17E2B00D06EE77D4F9D
:105B80003B78002B00D049E18020814A9368834311
:105B90009360804B9A68114399607F4B1B78DBB20E
:105BA000002B00D15BE18021754AC90113680B43CA
:105BB00013607A4A1378DBB2002B00D055E1734AA8
:105BC000704E90460B2241460A70013A4A70F0220C
:105BD0008B70CB700A71EE3A4A713E2240468B714F
:105BE000CA716F490A68120E02720A68120CD2B2A8
:105BF00042720A68120AD2B282720A680C21D2B2C8
:105C0000C272614A1170674A337013745C4A664B02
:105C100011680B4013601023524AD1680B43D360C4
:105C20002023D1680B43D3600823D1680B43D36092
:105C300093694C4CDB00FBD543461B78DBB299469D
:105C40002360180000F0C6FA4B46002B18D001253F
:105C5000A3691B02FCD44246337801350133DBB221
:105C60003370D35C3F4ADBB2136042463378EDB207
:105C7000DBB2D35C5840C0B200F0ACFAA945E7D221
:105C8000384A93691B02DB0FFBD1364A1060327829
:105C90000132D2B23270354A1370384A136002337F
:105CA0003B70F8E6C0213F4D314F2B7C5B00FB5A27
:105CB000194000D07CE02D4E3378DBB2581CC0B2C6
:105CC00030706846C0795B00D8532B7C5B00DB5B8F
:105CD000002B00D1C2E62B7C5B00D85B2B7C347898
:105CE00002331B18DBB2A34200D0B7E633782F4C47
:105CF000DBB2581CC0B2307080205B008000D853EB
:105D0000337800205B00D95313685B005B08136095
:105D10002B7C00225B00DB5B002398462B7C4344FA
:105D2000DBB25B00FB5ADBB2A354A35C5840C0B2A9
:105D300000F050FA43460133DBB298462B7C4246D2
:105D40005B00FB5A01334345E8DA0A4F3B78DBB28C
:105D5000022B00D18EE0032B00D07FE60022074B00
:105D60001A607BE60000154090070020980700208D
:105D700088050020A4070020480400209C0700207C
:105D80007C050020A0070020EC0200204C0400202D
:105D900000400050C04000501D0300204904002076
:105DA000B402002030020020FFFFFFFB4803002068
:105DB00013685B005B0813602B7CB34A013BDBB2CA
:105DC0001370137800225B00DA5364E6AE4A813424
:105DD0001378DBB2581CC0B21070AC485B001C5288
:105DE00013785B00195280211378A94ADBB213742F
:105DF000A84A090613680B4313604CE60022A64B21
:105E00001A6048E6A24AA54910740A68501C086046
:105E1000632A00D922E6A04A13601FE63B78022BD2
:105E200000D038E600F0B4F900239D4D9A4C9D490E
:105E300028703B70236023685A1C22608B42FAD979
:105E4000002323602B78002B00D024E60F22964BF2
:105E50001B68DBB22B702B7813402B701BE60621DE
:105E6000924A1170924A1370A3E61378013BDBB299
:105E7000137010E6002857D12379702B5CD023795A
:105E8000722B00D1CCE0217822786378C9B201333B
:105E90009A4200DCE2E563780133DBB22B742A7CA2
:105EA00023789B1ADBB223700129E5D9012302393B
:105EB000C9B202312A7CD218A25CD2B2E2540133B8
:105EC0009942F7D1D8E701233B60E4E53D60280023
:105ED000013500F07FF9EBB29A4601239946BB6980
:105EE000744D1B02FBD4424633780133DBB233706E
:105EF000D35CDBB22B603378DBB2D35C5840C0B2EA
:105F000000F068F94B460133DBB299469A45E6D179
:105F1000AB691B02DB0FFBD1664A1060327801329D
:105F2000D2B232702360B6E50023FF223B705C4B97
:105F30001A70B0E53B60AEE5002057495A4D086045
:105F4000627A2B681B0E9A4200D087E5A37AFF2263
:105F50009C462B681B0C13409C4500D07EE5E37AE1
:105F60009C462B681B0A13409C4500D076E5237B9A
:105F70009C462B6813409C4500D06FE503233B7083
:105F800063794D4CDBB223702378DBB2834277D048
:105F900008603378494ADBB21370494B494A1968A3
:105FA0000A4049491A604A79920765D58026474ACE
:105FB000474D1070AC68B443AC60464D403EAC6891
:105FC0003443AC60444C207038480478052C50D0E1
:105FD0000624047000243648047010244879A04335
:105FE00048710420497901423DD090253B4CA1687D
:105FF000A943A1601278002A00D12FE50022384978
:106000000A801C68374921401960374908602849CF
:106010000A7036490A701968354A0A401A601DE547
:1060200000201D4B20491860627A0B681B0E9A42B3
:1060300000D013E5FF22A57A0B681B0C13409D428C
:1060400000D00BE5E57A0B681B0A13409D4200D097
:1060500004E5247B0B6813409C4200D0FEE4104B07
:1060600038701A7017E590211C4A93680B439360AF
:10607000F4E402340470ADE70120144A1070ACE778
:106080003B70074B1A7006E5980700208805002032
:1060900030020020900700209C070020CC02002046
:1060A00049040020FFFF0F00B4020020AE020020D0
:1060B000860500200000154048040020A5070020A8
:1060C0007C050020FFFFFBFFF00200201D030020E5
:1060D00000400050C0400050740500208040005037
:1060E000B0020020FFFFFFBF00E100E082050020BA
:1060F000FFFFBFDF10B5FAF73DFEFDF773FC10BDE3
:1061000010B51C4A13695B075B0F052B1CD8022BCB
:106110001BD10123146A2404A40FA3429B415B42B8
:10612000E41A136A1B0323D4134B124A106A116A30
:10613000C005C00D8904C90E02305843023102F077
:1061400041F9E0400D4C03E004230C4C9B00E05867
:10615000084B99690907090F013102F033F9084B1F
:1061600060619C460749604402F02CF9A06110BDB3
:10617000054BDAE700020050001BB700E4000020E6
:1061800020A1070040420F00008051017047C04627
:106190000F200E4B1A7819785200D2B24A405200A2
:1061A0001978D2B24A4012011978D2B24A4019780D
:1061B000D20949005218D2B21A701B78044A18400A
:1061C0001378C0181F231840107070475005002026
:1061D000B20200200022C30700D55E32830701D53A
:1061E000BC235A40430701D561235A40030701D518
:1061F000C2235A40C30601D59D235A40830601D5C8
:1062000023235A40430601D546235A4043B2002B6C
:1062100001DA8C235A4010007047C046F0B544465E
:106220005F4656464D46F0B4C64BC74C98461A7862
:10623000237897B09A423DD02378002B41D1C34FA9
:10624000FF33FF33FA5AFE3B19009A4208D02378F5
:10625000DBB25A1CD2B222705B00FB5A8B42F6D1E1
:106260008021237849005B00FB5A9BB21A1E8A42A8
:1062700008D123780133DBB2237023785B00FB5A0B
:106280009342F6D023785B00FB5A002B12D0237880
:106290005B00DB5BDBB203930233DBB21A00944694
:1062A000029323786344DBB25B00DA5B80239B00BC
:1062B0009A4219D017B03CBC90469946A246AB46CC
:1062C000F0BD80212378A14F013B5B00FB5A4900C0
:1062D0008B42C5D02378DBB25A1CD2B222705B004D
:1062E000FB5A8B42F6D1BBE7002261462378634418
:1062F000DBB25B00DA53002901D101F0C3FB039B41
:1063000006AE0133DBB2013399463500B1444E4647
:106310000020A9462278D2B2511CC9B22170520085
:10632000BA5AD3B22B704340D8B20135FFF752FFAF
:10633000B542EFD1237880220133DBB22370844B46
:106340004E4699461B68D20413434A461360814B5C
:10635000B2789B46002804D01B789A4201D101F004
:10636000E3FA5B461B78934200D18AE05B461F78D4
:10637000FBB20193934200D19FE0002A62D13379AE
:10638000033BDBB22E2B5DD8734A9B00D3589F464C
:106390000422724B1A60724B033A1A70714B1B88BD
:1063A000C72B01D901F08CFA802140206E4A9368F6
:1063B0000B4393606D4A93688343936000226C4B58
:1063C0001A706C4B05321A704B466B4A1170196883
:1063D0006A4B0B4049460B60FA21694B4900196032
:1063E000684C694D2378DBB2591CC9B22170052174
:1063F000E9542378DBB2591CC9B221700421E95455
:106400002378DBB2591CC9B221700021E9542178EC
:10641000C9B24B1CDBB223705C4B1878C0B2471C6E
:10642000FFB21F7068542378DBB2591CC9B22170C7
:10643000B021E9542378DBB2591CC9B2217012781B
:10644000D2B2EA547178337801318B4200DCE6E055
:10645000C9B25B1A3370029B012B0CD9039A881CBA
:1064600094464B1C6044F318301849421A785A5429
:1064700001338342FAD15B46B2781B78934200D055
:1064800074E7434B31791B7801338B420CD0404B7E
:1064900040481B78DBB20370002905D03E4B1868DA
:1064A000012303433C480360394B19705B461F7856
:1064B000FBB20193934200D05FE74B4680221B68FA
:1064C000D20413434A4613607179712900D973E1EC
:1064D000324A8B00D3589F468021234A93688B43CE
:1064E00093604023214A91680B43936000221C4B28
:1064F0001A70204B1A78052A01D101F0EBF9062217
:106500001A7000214B4681201B4A800511701B68C0
:106510001C4C03434846036023781B4DDBB2581CD8
:10652000C0B220700520E8542378DBB2581CC0B2FA
:1065300020700420E8542378DBB2581CC0B22070CD
:1065400064E7C04698070020A507002088050020C2
:106550007C05002048040020708F000000E100E06E
:10656000740500208405002000400050C040005009
:1065700082050020AE02002086050020FFFFBFDF5D
:10658000E0020020EC0200204C0400204D05002019
:106590007505002094070020900700202C90000033
:1065A0008021E64A93688B4393604023E44A9068D5
:1065B00003439360FA220020E24B92001A80E24AE1
:1065C0004B46107081221B68920513434A461360A4
:1065D0008022DE4B92015A50DD4BDE4A1870DE4BB2
:1065E0007F311A60DD4A11701A68002AFCD1DC4B39
:1065F0001A70FAF7BFFB0323DA4A11680B431360E2
:10660000D94ADA4B1A60A0220123D20591680B43C4
:1066100093607178337801318B4200DD18E74B4687
:106620001A68D34B13404A46136043E6D14AD24B13
:1066300011680B40136005E78021CE4AC902136838
:106640000B431360CD4B1B78002B01D101F02FF9C8
:10665000CB4B1B88C72B01D901F029F980214020A1
:10666000B64A93680B439360B54A9368834393603B
:106670000022C44B1A70C44B05321A704B46B24A02
:1066800011701A68C14B13404A461360FA22B24B8C
:1066900052001A60D6E6F279002A01D001F08FF993
:1066A000BB4CBC4D2378DBB2591CC9B221701221FE
:1066B000E9542378DBB2591CC9B221701121E95485
:1066C0002378DBB2591CC9B22170EA542178CBB2CD
:1066D000694698460133DBB22370A14B1878C0B2EB
:1066E000471C0F740F7C1F704346E8542378DBB2BD
:1066F000591CC9B221709521E9542378DBB2591C89
:10670000C9B22170EA542378DBB2591CC9B2217096
:10671000EA542378DBB25A1CD2B222700B22EA541C
:106720002378DBB25A1CD2B222704222EA54237878
:10673000DBB2591CC9B221706921E9542378DBB25C
:10674000581CC0B220704420E8542378DBB2581C97
:10675000C0B22070E9542378DBB2591CC9B2217051
:106760006F21EA542378DBB25A1CD2B22270E9546A
:106770002378DBB25A1CD2B22270E9542378DBB200
:106780005A1CD2B222707322EA542378DBB25A1C0C
:10679000D2B222707422EA542378DBB25A1CD2B2ED
:1067A00022706522EA542378DBB25A1CD2B22270DE
:1067B0007222EA54019AE0E5019ADEE5B279764B5D
:1067C0001A70F2795A70327A9A70727ADA70019A83
:1067D000D3E5B279092A01D901F015FDF3790493C3
:1067E000303BDBB29A46012A11D93000911EC9B262
:1067F0000131019F71189C001B195B00047A303B2A
:106800001B190130DBB28142F5D19A4601975346FC
:10681000072B01D101F0F0FC604B98465C4C5D4DBC
:106820002378DBB2591CC9B2217011000931C9B2F9
:10683000E9542378DBB2591CC9B221701100083128
:10684000C9B2E9542378DBB2591CC9B221700021C6
:10685000E9542178CBB2694600930133DBB223704F
:106860003F4B1878C0B2471CCF75CF7D1F70009B7F
:10687000E8542378DBB2591CC9B221709321E95442
:106880002378DBB2591CC9B22170EA54002A14D013
:10689000531EDBB2083308A9F318019F02E00A78FF
:1068A000013104922278D2B2501CC0B220706846E6
:1068B000007CA8548B42F2D1019723786421DBB28B
:1068C0005A1CD2B222700322EA5423785246DBB219
:1068D0001F000133DBB223704346985CC0B201F065
:1068E00071FD03003033DBB25246EB554346985CF2
:1068F0006421C0B201F0ECFDCBB29A4623780A21A4
:10690000DBB298460133DBB22370504601F05AFDEA
:10691000030042463033DBB2AB5423780A21DBB2AA
:1069200098460133DBB22370504601F0D1FD0B00D5
:1069300042463033DBB2AB54019A1EE500400050B2
:10694000C0400050E40200208605002000E100E085
:10695000A4070020DC050000E0020020490400201C
:106960004D05002000C000500400FA050CED00E0C9
:10697000FFFFFFFB90070020FFFFFBFF1D03002030
:106980008405002082050020AE020020FFFFBFDF4B
:10699000EC0200204C040020E8020020F00200205D
:1069A000B179092901D901F02EFC7318DA79092A85
:1069B00001D901F028FCDB4CDB4D2078C0B2431C30
:1069C000DBB223708B18DBB29F1DFFB22F542078EF
:1069D0000533C0B2471CFFB2DBB227702B542378BB
:1069E000DBB2581CC0B220700020E8542078C3B23B
:1069F00098460133DBB22370CC4B1F78F8B26F4658
:106A00008246013038713879187043465046E85450
:106A10002378DBB2581CC0B220709320E85423784E
:106A2000DBB2581CC0B22070E954002910D006AB6C
:106A3000D81D4B1EDBB20833F3189C462778FFB2F3
:106A40007B1CDBB2237003780130EB558445F5D114
:106A50002378DBB2581CC0B22070EA54002A01D15E
:106A600001F0D9FB571EFFB2B8460F000B000937E3
:106A700047440833B8469C46F018B0442778FFB224
:106A80007B1CDBB2237003780130EB554045F5D118
:106A9000F4796346303CE4B201290DD93700012571
:106AA000A000201840003C7A303801350019EDB2C2
:106AB000C4B20137A942F3D8F55C303DEDB2012AEA
:106AC00012D9023AD2B20232591CD3182A007118D4
:106AD000F3189000121852000878303A1218013159
:106AE000D2B29942F5D11500601EC0B22900FAF762
:106AF00051F9072C01D101F03DFBB2783DE44B4642
:106B00001A688B4B874C13404A4613602378864D96
:106B1000DBB25A1CD2B222700522EA542378DBB2CF
:106B20005A1CD2B222700422EA542378DBB25A1CD7
:106B3000D2B222700022EA5490466A462178C9B245
:106B40004B1CDBB22370794B1878C0B2471C17740A
:106B5000177C1F7068542378DBB2591CC9B22170AE
:106B600094214246E9542378DBB2591CC9B2217002
:106B7000EA54019AFFF701FC6E49707A0B68019A9A
:106B80001B0E984201D0FFF7F8FBFF200B68B47A88
:106B90001B0C03409C4201D0FFF7EFFB0B68F47A1B
:106BA0001B0A03409C4201D0FFF7E7FB0B68317BD7
:106BB0000340994201D0FFF7E0FB4B4680211B6860
:106BC00089040B434946574C0B602378564DDBB282
:106BD000591CC9B221700521E9542378DBB2591C34
:106BE000C9B221700421E9542378DBB2591CC9B21F
:106BF00021700021E9542178C9B24B1CDBB223700B
:106C00004A4B1878C0B2471CFFB21F7068542378F3
:106C1000DBB2591CC9B221709421E9542378DBB24C
:106C2000591CC9B221700121E954FFF7A6FB3D4C64
:106C30003D4D23786946DBB25A1CD2B2227006223F
:106C4000EA542378DBB25A1CD2B222700522EA54ED
:106C50002378DBB25A1CD2B222700022EA5490464A
:106C60002278D2B2531CDBB22370304B1878C0B2FA
:106C7000471C0F740F7C1F70A8542378DBB25A1C7A
:106C8000D2B222709022EA542278D2B2531CDBB2E4
:106C90002370B379AB54142B01D101F079FA01D8E8
:106CA00001F0F9F9192B01D101F0E4F901D801F053
:106CB000ADF91C2B01D101F099F9FE2B01D101F0A6
:106CC0007FF91A2B01D101F062F92378DBB25A1C4B
:106CD000D2B222700022EA54019AFFF74EFBB37938
:106CE000152B01D101F013F901D801F0FDF81A2B91
:106CF00001D101F0D9F801D901F0C7F8172B01D162
:106D000001F0BCF801D201F0B2F8182B01D101F06A
:106D1000A7F8192B12D10D23074A0E2113700093E7
:106D200011E0C046EC0200204C0400204D0500207C
:106D3000FFFFFFFDB402002064020020F04A137838
:106D4000591C0093C9B206276846EE4C2378DBB283
:106D50005D1CEDB22570EC4DEF542378DBB25F1C67
:106D60000774FFB227700527EF542378DBB25F1C4E
:106D70000774FFB227700027EF542378DBB29C46DC
:106D80000133DBB22370E14B1F78FFB2B846012715
:106D900047440774077C1F7063464746EF54009BC7
:106DA000112B01D901F045F89800D94B1B589F468B
:106DB000B379002B00D0FFE4737A019A3E2B01D007
:106DC000FFF7DBFAD349B07A0B681B0E984201D06B
:106DD000FFF7D3FAFF200B68F47A1B0C03409C42A8
:106DE00001D0FFF7CAFA0B68347B1B0A03409C42B0
:106DF00001D0FFF7C2FA0B68717B1840814201D0C5
:106E0000FFF7BBFAF9F7B6FFF9F79CFFF82040024D
:106E1000F9F76EFF5B461B78BF4AC04C1B02134359
:106E200023602168BE48F9F70DFF0323BD4A1168AE
:106E30000B43236023681360BB4ABC4B1A60FEE718
:106E4000BB4BB04C1B685B0301D500F0BAFDAE4DE7
:106E5000AE4B2278D2B2511CC9B221700521A9547F
:106E60002278D2B2511CC9B221700421A9542178D0
:106E7000C9B24A1CD2B2227000226A5490466A46B5
:106E80002178C9B2481CC0B220701878C0B2471C23
:106E90001774177C42461F7068542378DBB2591C64
:106EA000C9B221709221E9542378DBB2591CC9B2CE
:106EB00021701221E954924B1A70019AFFF75DFA82
:106EC000904C914D2378DBB25A1CD2B2227006222C
:106ED000EA542378DBB25A1CD2B222700522EA545B
:106EE0002378DBB25A1CD2B222700022EA549046B8
:106EF0006A462178C9B24B1CDBB22370834B1878E9
:106F0000C0B2471C1774177C42461F706854237820
:106F1000DBB2591CC9B221708621E9542378DBB257
:106F2000591CC9B22170EA542378DBB2591CC9B28A
:106F30002170EA54019AFFF720FA724C724D2378BF
:106F4000DBB25A1CD2B222700522EA542378DBB29B
:106F50005A1CD2B222700422EA542378DBB25A1CA3
:106F6000D2B222700022EA542278D2B2531CDBB291
:106F70002370664B1978C9B2481CC0B21870A95466
:106F80002378DBB25A1CD2B222708B22EA542378C7
:106F9000DBB25A1CD2B22270FF22EA54019AFFF7E8
:106FA000ECF9584C584D2378DBB25A1CD2B22270FF
:106FB0000522EA542378DBB25A1CD2B22270042292
:106FC000EA542378DBB25A1CD2B222700022EA546F
:106FD0002278D2B2531CDBB223704C4B1978C9B261
:106FE000481CC0B21870A9542378DBB25A1CD2B224
:106FF00022708822EA542378DBB25A1CD2B2227063
:107000000122EA54019AFFF7B8F93E4C3E4D23782D
:10701000DBB25A1CD2B222700522EA542378DBB2CA
:107020005A1CD2B222700422EA542378DBB25A1CD2
:10703000D2B222700022EA542278D2B2531CDBB2C0
:107040002370324B1978C9B2481CC0B21870A954C9
:107050002378DBB25A1CD2B222708A22EA542378F7
:10706000DBB25A1CD2B222708022EA54019AFFF796
:1070700084F980202F4A93688343936040232E4AEB
:1070800091680B439360FA2200212C4B92001A80E6
:107090002B4A4B46117081221B68920513434A46C6
:1070A0001360234A274B1468234013609023264A19
:1070B0009468234393608022244B92011A50244BFE
:1070C000244A1970244BFF311A60244A11701A683F
:1070D000002AFCD10D4B1A70F9F74CFE0323114A1C
:1070E00011680B431360104A104B1A60A022012351
:1070F000D20591680B439360B278FFF73EF9C04622
:1071000064020020EC0200204C0400204D05002009
:10711000F4910000B40200203E00FFFFD0020020E6
:107120001CF0010000C000500400FA050CED00E066
:107130009007002000400050C0400050E4020020B2
:1071400086050020FFFFFBFF8040005000E100E0CB
:10715000A4070020DC050000E00200204904002014
:107160008021F74A890213680B4201D100F05DFCCF
:107170007F201168F34B0B40F34913600B780340F9
:107180000B70F24CF24D2378DBB2591CC9B221705E
:107190000521E9542378DBB2591CC9B221700421BE
:1071A000E9542378DBB2591CC9B221700021E9549B
:1071B0002178CBB2694698460133DBB22370E54BA8
:1071C0001878C0B2471C0F740F7C1F704346E854F8
:1071D0002378DBB2591CC9B221708721E954217888
:1071E000C9B24B1CDBB223701368019A9B03DB0FFF
:1071F0006B54FFF7C2F8D54CD54D2378DBB25A1C3F
:10720000D2B222700522EA542378DBB25A1CD2B2E1
:1072100022700422EA542378DBB25A1CD2B22270C4
:107220000022EA542278D2B2531CDBB22370C94B3D
:107230001978C9B2481CC0B21870A9542378DBB2BF
:107240005A1CD2B222708222EA542378DBB25A1C32
:10725000D2B22270B279EA54019AFFF78EF8BB4C91
:10726000BB4D2378DBB25A1CD2B222700722EA54FB
:107270002378DBB25A1CD2B222700622EA54237859
:10728000DBB25A1CD2B222700022EA5490466A46FF
:107290002178C9B24B1CDBB22370AE4B1878C0B258
:1072A000471C1774177C1F7068542378DBB2591C75
:1072B000C9B221708521E9542378DBB2591CC9B2C7
:1072C00021700C21E9542378DBB2591CC9B221701A
:1072D000012146E49D4C9E4D2378DBB25A1CD2B26C
:1072E00022700B22EA542378DBB25A1CD2B22270ED
:1072F0000A22EA542378DBB25A1CD2B2227000224E
:10730000EA5490466A462178C9B24B1CDBB223701E
:10731000904B1878C0B2471C1774177C42461F70F8
:1073200068542378DBB2591CC9B221708421E95416
:107330002378DBB2591CC9B221700121E9542378AA
:10734000DBB2591CC9B22170EA542378DBB25A1C53
:10735000D2B222703E22EA542378DBB25A1CD2B257
:1073600022707D4A1168090EE9542178C9B24B1C7C
:10737000DBB2237013681B0CDBB26B542178C9B2EB
:107380004B1CDBB2237013681B0ADBB26B542378EF
:10739000DBB2591CC9B221701268D2B2EA54019A08
:1073A000FEF7EBFF6D4A694C694D2378DBB2591C3F
:1073B000C9B221700F21E9542378DBB2591CC9B23C
:1073C00021700421E9542378DBB2591CC9B2217021
:1073D0000021E95488462178CBB269469A460133A8
:1073E000DBB223705B4B1878C0B2471C0F740F7C64
:1073F00051461F7068542178C9B2481CC0B2207031
:10740000B02068542178C9B2481CC0B220701078EE
:10741000C0B268542178C9B2481CC0B2207009209B
:1074200068542178C9B2481CC0B2207040466854E4
:107430002178C9B28846481C6946C0B220701878C5
:10744000C0B2471C0F740F7C1F704346E85423786A
:10745000DBB2591CC9B22170B221E9542378DBB2E6
:10746000591CC9B221700121E9542178C9B24B1CC1
:10747000DBB223701278002352B2002A05DA384BAF
:107480005B789A00D3185B00DBB26B542378DBB2D5
:107490005A1CD2B222700022EA542378DBB2591C63
:1074A000C9B22170EA542378DBB2591CC9B22170E9
:1074B0000221E95438E504222A4B1A602A4B033A88
:1074C0001A702A4B1B88C72B00D8B8E2234A1F4CDE
:1074D0001F4D2378DBB2591CC9B221700521E95434
:1074E0002378DBB2591CC9B221700421E9542378F6
:1074F000DBB2591CC9B221700021E9542178CBB20A
:10750000694698460133DBB22370124B1878C0B23B
:10751000471C0F740F7C1F704346E8542378DBB27E
:10752000591CC9B22170B021E9542378DBB2591C2F
:10753000C9B221701278D2B2EA54019AFEF71DFF47
:1075400090070020FFFFFDFFAE020020EC020020AC
:107550004C0400204D050020B402002086050020C8
:10756000F002002000E100E0740500208405002006
:107570008021DA4A93688B4393604023D84A91680C
:107580000B4393600022D74B1A70D74B1A78052A09
:1075900000D18BE206221A700023D44A8121137095
:1075A0004B461B6889050B4349460B60FBE6D04AF6
:1075B000D04B11680B401360019AFEF7DEFE0422E7
:1075C0008021CD4BC9021A60C94A13680B4313606E
:1075D000CA4B1B78002B00D1E7E1C94B1B88C72B96
:1075E00000D9E2E180214020BC4A93680B439360BC
:1075F000BB4A9368834393600022C24B1A70BA4B14
:1076000005321A704B46B94A11701A68BE4B1340C6
:107610004A461360FA22BD4B52001A60019AFEF7E7
:10762000ACFEBB4CBB4D2378DBB25A1CD2B22270ED
:107630000622EA542378DBB25A1CD2B22270052209
:10764000EA5423789446DBB25A1CD2B2227000224C
:10765000EA5490462278D2B2531CDBB22370AE4B70
:107660001978C9B2481CC0B21870A9542378DBB28B
:107670005A1CD2B222708322EA542378DBB25A1CFD
:10768000D2B222706246EA542378DBB25A1CD2B2DC
:1076900022704246EA54019AFEF76FFE9C4C9D4DC3
:1076A0002378DBB25A1CD2B222700622EA54237825
:1076B000DBB25A1CD2B222700522EA542378DBB224
:1076C0005A1CD2B222700022EA542378DBB2591C31
:1076D000C9B22170EA542378DBB2591CC9B22170B7
:1076E0008121E9542378DBB2591CC9B22170FE21F3
:1076F000E9542378DBB2591CC9B22170AF21E95497
:10770000854BAE391970854B1A70854B1A70784AC3
:1077100013688B431360794B019A1B78002B01D1BE
:10772000FEF72BFE4B4680211B68C9010B434946DF
:107730000B60FEF722FE764C764D2378DBB25A1CA6
:10774000D2B222700422EA542378DBB25A1CD2B29D
:1077500022700322EA542378DBB25A1CD2B2227080
:107760000022EA542278D2B2531CDBB223706A4B57
:107770001978C9B2481CC0B21870A9542378DBB27A
:107780005A1CD2B22270F122EA54019AFEF7F5FD9A
:10779000317A002900D187E106AB624A9C46092074
:1077A00014004B1EDBB20A33019F6044F3180578C6
:1077B0000130257001349842F9D1019700235354C8
:1077C0004B4901330868F371033303430B60002313
:1077D000019F03E00133182B00D14DE1985CD9B231
:1077E0000028F7D1CB1DDBB29C46881D0197C0B2A3
:1077F0006746474C2378DBB25D1CEDB22570454DE2
:10780000EF542378DBB25F1C98466B461F741F7CD5
:1078100043462770E8542378DBB2581CC0B220706E
:107820000020E85482462078C3B200930133DBB2D3
:107830002370394B68461F78FFB2BC460127674466
:107840000774077C00981F7063462B542378DBB2C3
:10785000581CC0B220709520E8542378DBB2581C25
:10786000C0B220705046E8542378DBB2581CC0B236
:1078700020700120E8542378DBB2581CC0B220707D
:10788000E954002901D1FEF797FF4B1EDBB201330B
:10789000019F9B182178C9B2481CC0B22070107893
:1078A000013268549342F5D13A00FEF766FD4B462B
:1078B00080221B68D20113434A461360FEF7C2FDC3
:1078C0004B4680221B68D20113434A461360074A85
:1078D000FEF786FD02321A70FEF713FE00400050DC
:1078E000C040005074050020AE0200208605002034
:1078F00090070020FFFFFBFF00E100E01D030020D8
:107900008405002082050020FFFFBFDFE002002089
:10791000EC0200204C0400204D05002094070020BC
:10792000750500205C05002000210624F04B19702D
:107930001878C0B2421CD2B21A70EE4A14541878A9
:10794000C0B2441CE4B21C70052414541878C0B2B0
:10795000441CE4B21C7011541878C0B2441CE4B248
:107960001C70E54CA44667462478E4B2651CEDB271
:107970003D7014541878C0B2441CE4B21C708624C4
:1079800014541878C0B2441CE4B21C70022414547D
:107990001878C0B2441CE4B21C70337913544346C7
:1079A0001970D64B1960FEF73AFE4B4680221B68D1
:1079B000D20113434A461360019AFEF7DEFCD04A17
:1079C00005E72378CB4DDBB25A1CD2B222700522D8
:1079D000EA542378DBB25A1CD2B222700422EA5451
:1079E0002378DBB25A1CD2B222700022EA542278E9
:1079F000D2B2531CDBB22370BF4B1978C9B2481CFA
:107A0000C0B21870A9542278D2B2511CC9B22170E8
:107A1000B021A9542178C9B24A1CD2B22270B94A05
:107A20001278D2B26A54FFF714FA13680B4313604A
:107A30008023B549087803430B70FFF7A2FB802130
:107A40004020B24A93680B439360B14A93688343E2
:107A500093600022AF4B1A70AA4AAB4B11707B396E
:107A600019704B461968AC4B0B4049460B60FA2124
:107A7000AA4B490019602AE5073301971E209C464E
:107A80001821B5E6237880220133DBB22370A44BA2
:107A9000D20499461B6806AE13434A461360A14BB5
:107AA000B2789B46FEF75DFC954A87E602321A7073
:107AB00072E52378DBB2581CC0B220709020E854E5
:107AC0002378DBB2581CC0B220701C20E854237805
:107AD000DBB2581CC0B220709348807CC0B2E8541E
:107AE0001170019AFEF749FC2378DBB2581CC0B232
:107AF00020709020E8542378DBB2581CC0B220706C
:107B00000C20E8542378DBB2581CC0B220708648A1
:107B1000C07CC0B2E854E3E72378DBB2581CC0B2A3
:107B200020709020E8542378DBB2581CC0B220703B
:107B30000B20E8542378DBB2581CC0B220707A487E
:107B40004079C009E854CBE72378DBB2581CC0B2B7
:107B500020709020E8542378DBB2581CC0B220700B
:107B60001920E8542078C0B2431CDBB223706E4B5E
:107B70005B795B06DB0F2B54B2E72378DBB2581C32
:107B8000C0B220709020E8542378DBB2581CC0B2F9
:107B900020701820E8542378DBB2581CC0B2207043
:107BA0000120E8549CE72378DBB2581CC0B2207057
:107BB0009020E8542378DBB2581CC0B22070FC201F
:107BC000E8542378DBB2581CC0B220701820E85467
:107BD00086E72378DBB2581CC0B220709020E854AE
:107BE0002378DBB2581CC0B22070FD20E854237803
:107BF000DBB2581CC0B220700820E85470E723782C
:107C0000DBB2581CC0B220709020E8542378DBB25D
:107C1000581CC0B220701A20E8542078C0B2431C0F
:107C2000DBB22370404B5B799B07DB0F2B5457E78C
:107C30002378DBB2581CC0B220709020E85423781F
:107C4000DBB2581CC0B220701720E8542378DBB296
:107C5000581CC0B2207034488079C0B2E8543FE765
:107C60002378DBB2581CC0B220709020E8542378EF
:107C7000DBB2581CC0B220701620E8542A4B1B7986
:107C8000DBB2032B00D18AE0042B00D17FE0022B72
:107C900000D025E72378DBB2581CC0B220708B20BF
:107CA000E8541DE72378DBB2581CC0B22070902046
:107CB000E8542378DBB2581CC0B22070152069E765
:107CC0002378DBB2581CC0B220709020E85423788F
:107CD000DBB2581CC0B220701420E8542378DBB209
:107CE000581CC0B220701048C078C0B2E854F7E603
:107CF000EC0200204C0400204D0500209C070020D1
:107D00005C05002086050020AE02002000400050E7
:107D1000C040005082050020FFFFBFDFE0020020CE
:107D20007C05002048040020F00200202378DBB20C
:107D3000581CC0B220709020E8542378DBB2581C45
:107D4000C0B220701320E8542378DBB2581CC0B2B4
:107D50002070E0488078C0B2E854C1E62378DBB2F6
:107D6000581CC0B220709020E8542378DBB2581C15
:107D7000C0B220701220E8542378DBB2581CC0B285
:107D800020700124D34840792040E854A8E62378A5
:107D9000DBB2581CC0B22070AA20E854A0E62378B9
:107DA000DBB2581CC0B220709B20E85498E62378C0
:107DB000DBB2581CC0B220709020E8542378DBB2AC
:107DC000581CC0B220701120E4E62378DBB2581CA6
:107DD000C0B220709020E8542378DBB2581CC0B2A7
:107DE00020701020E8542378DBB2581CC0B22070F9
:107DF000B8484078C0B2E85472E62378DBB2581C29
:107E0000C0B220709020E8542378DBB2581CC0B276
:107E100020700F20BEE62378DBB2581CC0B2207061
:107E20009020E8542378DBB2581CC0B22070FE20AA
:107E30007FE605202378043BE85404202378033BA5
:107E4000E8542378DBB2581CC0B220709120E8546B
:107E50002378DBB2581CC0B22070FF20E8543FE604
:107E60000C239D4A0D2113700093FEF76CFF07232E
:107E7000994A082113700093FEF765FF0823964A7C
:107E8000092113700093FEF75EFFFC2B25D019D952
:107E9000FD2B10D0FE2B01D0FEF750FF11238E4A90
:107EA00000931370FEF74FFF09238B4A0A211370CA
:107EB0000093FEF748FF0A23874A0B2113700093B3
:107EC000FEF741FF1C2B01D0FEF738FF1023824A3A
:107ED000112113700093FEF736FF0B237E4A0C210D
:107EE00013700093FEF72FFF102B3BD02BD9122BD2
:107EF00022D01AD3132B11D0142B01D0FEF71EFF62
:107F00000523754A062113700093FEF71CFF062314
:107F1000714A072113700093FEF715FF04236E4A80
:107F2000052113700093FEF70EFF02236A4A032116
:107F300013700093FEF707FF0323674A04211370B1
:107F40000093FEF700FF0C2B1AD00F2B11D00B2B38
:107F500001D0FEF7F3FE0E235F4A0F21137000934A
:107F6000FEF7F1FE01235C4A022113700093FEF735
:107F7000EAFE0023584A012113700093FEF7E3FE46
:107F80000F23554A102113700093FEF7DCFE514B6E
:107F9000F07998465B792278DBB2D2B2511CC9B233
:107FA000217000281DD001210224A9541C43210066
:107FB0000420F8F7EFFE4346019A5C71FEF7DDF905
:107FC0002278D2B2531CDBB223707F24F379AB54F6
:107FD000404A9046527914405A1E9341DB011C439B
:107FE000E5E7A854022293431C00E0E72378112020
:107FF000DBB25A1CD2B22270F4792100EC54F8F7AB
:10800000C9FE344B019A9C74FEF7B7F9162B1CD0AD
:10801000172B01D0FEF759FEF3799A46632B03D84C
:108020004346F37100239A4623785146DBB25A1C2B
:10803000D2B2227052460520EA54F8F7ABFE5246FF
:10804000244B9A71019AFEF798F9F379AA2B00D97B
:10805000C4E09A2B00D9B3E08B2302210320F371F3
:10806000F8F798FE1B4B98460223424613718B2269
:10807000FEF75AFF174BF07998465B792278DBB20E
:10808000D2B2511CC9B2217000281DD00121402458
:10809000A9541C438BE7102B47D030D80B2B1DD095
:1080A0000C2B01D0FEF711FE23781220DBB25A1CF4
:1080B000D2B22270F4792100EC54F8F76BFE054B34
:1080C000019ADC74FEF759F9A854402293431C002E
:1080D0006DE7C046F002002064020020584BF079A2
:1080E00098465B792278DBB2D2B2511CC9B22170BA
:1080F00000282AD001218024A9541C4357E7122BC1
:1081000027D0132B01D0FEF7E0FD23780120DBB24E
:108110005A1CD2B22270F4792100EC54F8F73AFEDE
:10812000474B019A9C70FEF728F923780020DBB2B8
:108130005A1CD2B22270F4792100EC54F8F72AFECE
:108140003F4B019A5C70FEF718F97F24A8541C403D
:108150002DE73B4BF07998465B792278DBB2D2B2BF
:10816000511CC9B2217000285ED001210124A954FC
:108170001C431CE73E2D01D0FEF7BFFC4B4680227E
:108180001B68120513434A461360B278FEF7F5F8F0
:10819000F3799A46FA2B02D9FA239A46F371237897
:1081A0005146DBB25A1CD2B2227052460220EA5427
:1081B000F8F7F0FD5246224BDA70019AFEF7DDF82F
:1081C0009B2303210320F371F8F7E4FD1C4B984631
:1081D0000323424613719B22FEF7A6FEAA23042125
:1081E0000320F371F8F7D6FD154B98460423424659
:1081F0001371AA22FEF798FE114B98460C234146B4
:10820000CB71FEF70BFB4B461A680E4B13404A46E8
:108210001360FEF704FAF479303CE4B2012908D97E
:108220000B000833FEF73AFCA854012293431C00CC
:10823000BDE671180D7A303DEDB2FEF755FCC04633
:10824000F0020020FFFFFFFDF0B5474680B406AC0A
:108250002678A0248027E405E5687F053D43E56096
:1082600090462B4DE2681540E560032423409C00B6
:108270000C23284D6A699A43130023436B61AB6951
:1082800034049C466246244B134023430124AB61D3
:10829000AB683B43AB60214B1D6A2C431C6200283A
:1082A00018D11C6A1E4820401862002919D00129E3
:1082B0001DD0022923D00C231849086A03430B62FE
:1082C000FF20424615494B6A83431A434A6204BC65
:1082D0009046F0BD8024186AE4002043186200290B
:1082E000E5D10C200D490B6A83430B62E8E70B488C
:1082F0000B31036A8B4308390B430362E0E70748FD
:108300000A31036A8B4304390B430362D8E7C04642
:10831000FFFFFFEF00020050FFFF00FF00000E40D4
:10832000FFFBFFFF10B51B4B1B6BDB0724D4194B66
:108330001B6B9B0712D4174B1B6B5B0700D410BD44
:10834000154A5369002B01D0D0689847072213497A
:108350000B689343033A13430B60F0E70E4A13692B
:10836000002B01D09068984707220C490B68934373
:10837000053A13430B60DEE7074A1368002B01D070
:1083800050689847072205490B689343063A134300
:108390000B60CCE700000E408802002030000E4049
:1083A000072206490B689343063A13430B6080216A
:1083B000034A0901136A0B431362704730000E40F1
:1083C00000000E40002243088B4274D303098B4205
:1083D0005FD3030A8B4244D3030B8B4228D3030C95
:1083E0008B420DD3FF22090212BA030C8B4202D337
:1083F0001212090265D0030B8B4219D300E0090A5F
:10840000C30B8B4201D3CB03C01A5241830B8B4267
:1084100001D38B03C01A5241430B8B4201D34B0350
:10842000C01A5241030B8B4201D30B03C01A5241B5
:10843000C30A8B4201D3CB02C01A5241830A8B423A
:1084400001D38B02C01A5241430A8B4201D34B0223
:10845000C01A5241030A8B4201D30B02C01A524187
:10846000CDD2C3098B4201D3CB01C01A524183093B
:108470008B4201D38B01C01A524143098B4201D375
:108480004B01C01A524103098B4201D30B01C01AA0
:108490005241C3088B4201D3CB00C01A524183081A
:1084A0008B4201D38B00C01A524143088B4201D347
:1084B0004B00C01A5241411A00D2014652411046A7
:1084C0007047FFE701B5002000F0F0F802BDC0469C
:1084D0000029F7D076E7704703460B437FD400228C
:1084E00043088B4274D303098B425FD3030A8B4248
:1084F00044D3030B8B4228D3030C8B420DD3FF22B2
:10850000090212BA030C8B4202D31212090265D07F
:10851000030B8B4219D300E0090AC30B8B4201D332
:10852000CB03C01A5241830B8B4201D38B03C01A79
:108530005241430B8B4201D34B03C01A5241030BF0
:108540008B4201D30B03C01A5241C30A8B4201D3A1
:10855000CB02C01A5241830A8B4201D38B02C01A4C
:108560005241430A8B4201D34B02C01A5241030AC3
:108570008B4201D30B02C01A5241CDD2C3098B42A8
:1085800001D3CB01C01A524183098B4201D38B0125
:10859000C01A524143098B4201D34B01C01A5241C8
:1085A00003098B4201D30B01C01A5241C3088B420D
:1085B00001D3CB00C01A524183088B4201D38B00F8
:1085C000C01A524143088B4201D34B00C01A52419A
:1085D000411A00D201465241104670475DE0CA0F71
:1085E00000D04942031000D34042534000229C4631
:1085F00003098B422DD3030A8B4212D3FC2289013B
:1086000012BA030A8B420CD3890192118B4208D310
:10861000890192118B4204D389013AD0921100E072
:108620008909C3098B4201D3CB01C01A5241830986
:108630008B4201D38B01C01A524143098B4201D3B3
:108640004B01C01A524103098B4201D30B01C01ADE
:108650005241C3088B4201D3CB00C01A5241830858
:108660008B4201D38B00C01A5241D9D243088B42AE
:1086700001D34B00C01A5241411A00D20146634651
:1086800052415B10104601D34042002B00D54942B5
:10869000704763465B1000D3404201B5002000F0F4
:1086A00005F802BD0029F8D016E770477047C046AC
:1086B0008407000092070000A0070000C607000022
:1086C000DC070000EA070000F807000006080000C9
:1086D0005E0700006C0700000000000020000000A2
:1086E0000000100020001000D2200000341A00000A
:1086F000C4200000C4200000C4200000C4200000EA
:10870000C4200000C4200000C4200000C4200000D9
:10871000C4200000C4200000C4200000C4200000C9
:10872000C4200000C4200000C4200000341A00004F
:10873000341A0000341A0000341A0000341A000001
:10874000341A0000341A0000341A0000341A0000F1
:10875000B4200000B4200000B4200000B4200000C9
:10876000B4200000B4200000B4200000341A00003F
:10877000A4200000A4200000A4200000341A00005F
:10878000341A0000341A0000341A0000341A0000B1
:10879000341A00009C200000942000006420000097
:1087A0005C2000003020000028200000341A000067
:1087B000341A0000341A0000341A0000341A000081
:1087C000341A0000341A0000341A0000341A000071
:1087D000341A0000341A0000341A0000341A000061
:1087E000341A000012200000FE1F0000F61F0000D7
:1087F000CE1F0000AC1F0000901F0000341A0000C4
:10880000341A0000341A0000341A0000341A000030
:10881000341A0000341A0000341A0000341A000020
:10882000341A0000341A0000341A0000341A000010
:10883000341A0000341A0000341A0000341A000000
:10884000341A0000341A0000341A0000341A0000F0
:10885000341A0000341A00007A1F00007A1F00004A
:108860007A1F00007A1F00007A1F00007A1F0000A4
:108870007A1F00007A1F00007A1F00007A1F000094
:10888000641F0000641F0000641F0000641F0000DC
:10889000641F0000641F0000641F0000641F0000CC
:1088A000641F0000641F00004E1F00004E1F0000E8
:1088B0004E1F00004E1F00004E1F00004E1F000004
:1088C0004E1F00004E1F00004E1F00004E1F0000F4
:1088D000341A0000341A0000341A0000341A000060
:1088E000341A0000341A0000341A0000341A000050
:108AC000341A00003E1F000030353A3F44494E54EE
:108AD000585C61666B707500A51264640381C80CF4
:108AE0003E041EFFFFFFFFFFFFFF0530FF000000F9
:108AF000AC280000C6280000DA280000EE2800009C
:108B000002290000062900000629000006290000AD
:108B10000629000006290000062900000629000099
:108B20000629000020290000322900004429000005
:108B300056290000682900007C29000090290000C7
:108B4000B2290000D6290000D6290000D62900004D
:108B5000D6290000F4290000F42900005E28000056
:108B6000502800009A280000582C0000EA2D000030
:108B7000FA2D0000DA2D00002A2E00000A2E000037
:108B80001A2E0000802C00003A2E00003A2E000021
:108B90003A2E00003A2E00003A2E00003A2E000035
:108BA0003A2E00003A2E0000A82C0000D22C000023
:108BB000002D00002A2D0000862D0000582D0000F9
:108BC000B02D00002A2C00009A2E0000B02E0000CC
:108BD000C62E0000DC2E0000F22E0000082F000040
:108BE0001E2F0000342F0000982E0000982E000049
:108BF000982E0000982E0000982E0000982E00005D
:108C0000982E0000982E00004A2F00005C2F0000D4
:108C10006E2F0000802F0000922F0000A42F000074
:108C2000B62F0000882E0000103000001030000029
:108C300010300000103000001A3000001A30000020
:108C40001A3000001A3000000E3000000E30000014
:108C50000E3000000E3000000E3000000E3000001C
:108C60000E3000000E3000002630000032300000D0
:108C70003E3000004A3000005630000062300000F4
:108C80006E30000004300000B6300000B630000046
:108C9000B6300000B6300000C8300000C830000018
:108CA000C8300000C8300000203100002031000032
:108CB0002031000020310000203100002031000070
:108CC0002031000020310000DA300000E4300000E4
:108CD000EE300000F8300000023100000C310000DE
:108CE00016310000AC300000723100007C31000011
:108CF000643100009E3100008A3100009431000090
:108D00004831000056310000E8310000F831000021
:108D1000083200001032000018320000203200003B
:108D2000D8310000C8310000CA320000CA32000049
:108D3000AA320000AA3200008A3200008A32000003
:108D4000CE320000CE320000923300008E3300009D
:108D50008A33000086330000823300003E33000077
:108D600072330000963300000E3400000E34000011
:108D70000034000000340000DE330000DE33000069
:108D800018340000183400007436000074360000F7
:108D9000743600007436000054360000543600006B
:108DA00054360000543600003234000032340000E3
:108DB000323400003234000032340000323400001B
:108DC0003234000032340000503600004C360000CF
:108DD0004836000044360000403600003C360000B3
:108DE0002C3600002234000028360000283600000F
:108DF000163600001636000032350000323500000D
:108E000094360000943600002E3800002E38000002
:108E10002A3800002A3800002638000026380000D2
:108E200034380000343800001237000012370000D8
:108E3000EA360000EA360000D2360000D2360000E2
:108E400002380000023800001C38000038380000EA
:108E5000903700001C380000E63700001C38000086
:108E60001C3800001C380000F23700001C380000DD
:108E70001C3800001C3800001C3800001C380000A2
:108E80001C3800001C380000EC3700008E39000050
:108E90008E3900007E3900007E3900006A390000FA
:108EA0006A390000A4390000A43900000204081047
:108EB0009A3A0000AC3A0000C23A0000DA3A0000E8
:108EC000E83A0000F63A0000043B0000123B0000C4
:108ED000203B0000323B0000763A00008C3A000054
:108EE0000100000002000000020000000400000079
:108EF000904700001C470000424700005247000016
:108F0000C0470000AC470000C6460000E246000033
:108F100064470000764700006A4700007C47000075
:108F20006A4700007C470000CC430000E647000091
:108F3000EC4700007C470000EC4700007C47000045
:108F4000CC430000E6470000D448000082490000FE
:108F5000D4480000CA480000EE480000FA4D000066
:108F6000A84C0000A84C0000F44F0000F44F000093
:108F7000386600002C660000446400004464000071
:108F80004464000044640000A065000044640000E4
:108F90004464000044640000446400004464000031
:108FA0004464000044640000446400004464000021
:108FB0004464000044640000446400004464000011
:108FC0004464000044640000446400004464000001
:108FD00044640000446400004464000044640000F1
:108FE00044640000446400004464000044640000E1
:108FF00044640000446400004464000044640000D1
:1090000044640000446400004464000044640000C0
:1090100044640000446400004464000044640000B0
:1090200044640000D864000090630000B86700004A
:109030009C76000022760000BE750000AE75000030
:10904000D47200005E720000F671000060710000D2
:10905000727000000A700000A26F00003A6F0000FA
:10906000B8670000C06E0000B06D0000406E0000E8
:109070003C6D0000DE6C00002E6C0000786B000080
:10908000FE6A0000A0690000D2670000BC67000013
:109090009666000090770000B8670000B86700008F
:1090A000B8670000B8670000B8670000B867000044
:1090B000B8670000B8670000B8670000B867000034
:1090C000B8670000B8670000B8670000B867000024
:1090D000B8670000B8670000B8670000B867000014
:1090E000B8670000B8670000B8670000707500003E
:1090F000B6740000A4730000B8670000B8670000F1
:10910000B8670000B8670000B8670000B8670000E3
:10911000B8670000B8670000B8670000B8670000D3
:10912000B8670000B8670000B8670000B8670000C3
:10913000B8670000B8670000B8670000B8670000B3
:10914000B8670000B8670000B8670000B8670000A3
:10915000B8670000B8670000B8670000B867000093
:10916000B8670000B8670000B8670000B867000083
:10917000B8670000B8670000B8670000B867000073
:10918000B8670000B8670000B8670000B867000063
:10919000B8670000B8670000B8670000B867000053
:1091A000B8670000B8670000B8670000B867000043
:1091B000B8670000B8670000B8670000B867000033
:1091C000B8670000B8670000B8670000B867000023
:1091D000B8670000B8670000B8670000B867000013
:1091E000B8670000B8670000B8670000B867000003
:1091F00036770000FA7D0000CA7D0000AE7D0000D9
:109200005C7D00002C7D0000C07C0000A47C000080
:10921000607C0000307C0000FE7B0000D27B000000
:10922000A67B00007A7B0000487B0000187B0000D2
:0C923000E87A0000B27A0000167E000010
:10923C00FF40404040404040334040403440353691
:10924C0040404040404040403A4040403B403C372A
:10925C00404040403F403D3840403E3940FB40405C
:10926C004040404040404040244040402340222168
:10927C00404040401F401E2040401D1C401B4040B1
:10928C00404040401940181A4040171640154040C5
:10929C004040251440134040403240404040404044
:1092AC004040404040404040FE4040400E400D0C8D
:1092BC00404040400A40090B4040080740064040EF
:1092CC004040404004400305404002014000404003
:1092DC0040400F1040114040401240404040404040
:1092EC0040404040FD402B3040402A2F4031404010
:1092FC004040292E402D4040402C404040404040B2
:10930C004040FA28402740404026404040404040E2
:10931C0040FC0000001BB700000000000080510161
:10932C001027000000805101008051011600000040
:00000001FF
